 sw_utilityG

 Timestamp is 548ff4a9 (Tue Dec 16 17:00:25 2014)

 Preferred load address is 00100000

 Start         Length     Name                   Class
 0001:00000000 00010430H .text                   CODE
 0001:00010430 000000c4H .text$yc                CODE
 0001:000104f4 00000074H .text$yd                CODE
 0002:00000000 00006bdcH .rdata                  DATA
 0002:00006bdc 000000e4H .xdata                  DATA
 0002:00006cc0 00000000H ATL$__a                 DATA
 0002:00006cc0 00000000H ATL$__z                 DATA
 0002:00006cc0 0000003cH .idata$2                DATA
 0002:00006cfc 00000014H .idata$3                DATA
 0002:00006d10 0000021cH .idata$4                DATA
 0002:00006f2c 00000024H .idata$6                DATA
 0002:00006f50 00001ca2H .edata                  DATA
 0003:00000000 0000021cH .idata$5                DATA
 0003:0000021c 00000004H .CRT$XCA                DATA
 0003:00000220 00000004H .CRT$XCAA               DATA
 0003:00000224 00000004H .CRT$XCL                DATA
 0003:00000228 00000010H .CRT$XCU                DATA
 0003:00000238 00000004H .CRT$XCZ                DATA
 0003:0000023c 00000004H .CRT$XIA                DATA
 0003:00000240 00000004H .CRT$XIZ                DATA
 0003:00000244 00000004H .CRT$XPA                DATA
 0003:00000248 00000004H .CRT$XPZ                DATA
 0003:0000024c 00000004H .CRT$XTA                DATA
 0003:00000250 00000004H .CRT$XTZ                DATA
 0003:00000254 00000078H .data                   DATA
 0003:000002d0 000028adH .bss                    DATA
 0004:00000000 00000a88H .pdata                  DATA
 0005:00000000 000000a0H .rsrc$01                DATA
 0005:000000a0 000003dcH .rsrc$02                DATA

  Address         Publics by Value              Rva+Base       Lib:Object

 0000:00000000       ___safe_se_handler_count   00000000     <absolute>
 0000:00000000       ___safe_se_handler_table   00000000     <absolute>
 0001:00000000       ??4CVerInfo@@QAAAAV0@ABV0@@Z 00101000 f i CVERINFO.obj
 0001:0000001c       ??1CVerInfo@@QAA@XZ        0010101c f   CVERINFO.obj
 0001:00000048       ?InitVerInfoStruct@CVerInfo@@AAAHPAG@Z 00101048 f   CVERINFO.obj
 0001:000000f8       ?GetProductVersionStr@CVerInfo@@QAAPAGXZ 001010f8 f   CVERINFO.obj
 0001:00000104       ?GetFileVersionStr@CVerInfo@@QAAPAGXZ 00101104 f   CVERINFO.obj
 0001:0000010c       ?GetProductNameStr@CVerInfo@@QAAPAGXZ 0010110c f   CVERINFO.obj
 0001:0000011c       ?GetVerResourceString@CVerInfo@@AAAPAGPAG@Z 0010111c f   CVERINFO.obj
 0001:000001b0       ?SetProductNameStr@CVerInfo@@AAAXXZ 001011b0 f   CVERINFO.obj
 0001:000001e0       ?SetFileVersionStr@CVerInfo@@AAAXXZ 001011e0 f   CVERINFO.obj
 0001:00000210       ?SetProductVersionStr@CVerInfo@@AAAXXZ 00101210 f   CVERINFO.obj
 0001:00000244       ?Init@CVerInfo@@AAAHPAG@Z  00101244 f   CVERINFO.obj
 0001:00000270       ?GetVerResourceStr@CVerInfo@@QAAPAGPAG@Z 00101270 f   CVERINFO.obj
 0001:000002a0       ??0CVerInfo@@QAA@XZ        001012a0 f   CVERINFO.obj
 0001:0000030c       ??0CVerInfo@@QAA@PAG@Z     0010130c f   CVERINFO.obj
 0001:00000348       ??0CVerInfo@@QAA@PAUHINSTANCE__@@@Z 00101348 f   CVERINFO.obj
 0001:000003b4       ??0SW_RegistryKey@@QAA@ABV0@@Z 001013b4 f i ModemStat.obj
 0001:000003d8       ??4SW_RegistryKey@@QAAAAV0@ABV0@@Z 001013d8 f i ModemStat.obj
 0001:000003f0       ?HKey@SW_RegistryKey@@IBAQAUHKEY__@@XZ 001013f0 f i ModemStat.obj
 0001:000003f8       ?HKey@SW_RegistryKey@@IAAQAUHKEY__@@QAU2@@Z 001013f8 f i ModemStat.obj
 0001:00000408       ?Buffer@SW_RegistryKey@@IBAPAXXZ 00101408 f i ModemStat.obj
 0001:00000410       ?Buffer@SW_RegistryKey@@IAAXPAX@Z 00101410 f i ModemStat.obj
 0001:00000418       ?IsOpen@SW_RegistryKey@@UAAHXZ 00101418 f i ModemStat.obj
 0001:0000042c       ??1SWISYNCBLOCK@@QAA@XZ    0010142c f i ModemStat.obj
 0001:00000438       ?SetMessageVars@CModemStatus@@SAXXZ 00101438 f i ModemStat.obj
 0001:00000584       ??0CModemStatus@@QAA@XZ    00101584 f   ModemStat.obj
 0001:000006c0       ?PrepareRilDevSpecificInfo@CModemStatus@@QAAPAUtagDEVSPECIFICDATA@@KKAAK@Z 001016c0 f   ModemStat.obj
 0001:0000084c       ?RILDeregister@CModemStatus@@QAAHXZ 0010184c f   ModemStat.obj
 0001:000008a8       ?UpdateCallTypeAndStatus@CModemStatus@@QAAKKKGAAH@Z 001018a8 f   ModemStat.obj
 0001:00000cd8       ?RilResultCallback@@YAXKJPBXKK@Z 00101cd8 f   ModemStat.obj
 0001:00001188       ?WAITFORCOMMANDCOMPLETION@@YAXK@Z 00102188 f i ModemStat.obj
 0001:000011cc       ?PROCESS_RESULT_WITH_PAYLOAD@@YAXKPAPAEPAKK@Z 001021cc f   ModemStat.obj
 0001:0000125c       ?ProcessErrorFunc@@YAHAAUtagErrorInfo@@@Z 0010225c f   ModemStat.obj
 0001:000013bc       ?ExecNoParamDevSpecificWithResponsePayload@@YAHKPAPAEPAKAAUtagErrorInfo@@@Z 001023bc f   ModemStat.obj
 0001:00001554       ?GetEquipmentState@@YAHAAUtagErrorInfo@@@Z 00102554 f   ModemStat.obj
 0001:000016a4       ?ModGetRegistrationStatus@@YAHAAUtagErrorInfo@@@Z 001026a4 f   ModemStat.obj
 0001:000017f4       ?ModGetCurrentSystemType@@YAHAAUtagErrorInfo@@@Z 001027f4 f   ModemStat.obj
 0001:00001944       ?ModGetCallList@@YAHAAUtagErrorInfo@@@Z 00102944 f   ModemStat.obj
 0001:00001a8c       ?ModGetPacketDataStatus@@YAHAAUtagErrorInfo@@@Z 00102a8c f   ModemStat.obj
 0001:00001b20       GetAdvancedMenuInfo        00102b20 f   ModemStat.obj
 0001:00001be0       GetProvisionInfo           00102be0 f   ModemStat.obj
 0001:00001d84       GetCarrierIndex            00102d84 f   ModemStat.obj
 0001:00001dc4       GetCallGuardRegistry       00102dc4 f   ModemStat.obj
 0001:00001df8       SetCallGuardRegistry       00102df8 f   ModemStat.obj
 0001:00001e28       GetActWizDisabledRegistry  00102e28 f   ModemStat.obj
 0001:00001e5c       SetActWizDisabledRegistry  00102e5c f   ModemStat.obj
 0001:00001e8c       GetLogoTestReg             00102e8c f   ModemStat.obj
 0001:00001ec0       IsConsumerProduct          00102ec0 f   ModemStat.obj
 0001:00001ef4       EnableCarrierLogo          00102ef4 f   ModemStat.obj
 0001:00001f24       SetAutoUpdateTime          00102f24 f   ModemStat.obj
 0001:00001f54       SetAutoUpdateTimeUI        00102f54 f   ModemStat.obj
 0001:00001f84       GetAutoUpdateTime          00102f84 f   ModemStat.obj
 0001:00001fb8       GetAutoUpdateTimeUI        00102fb8 f   ModemStat.obj
 0001:00001fec       ChangeCarrierIndex         00102fec f   ModemStat.obj
 0001:00002024       RepairPhoneBookRegKeys     00103024 f   ModemStat.obj
 0001:0000204c       GetRilTechHdrinfo          0010304c f   ModemStat.obj
 0001:000021e0       GetIOTAStatus              001031e0 f   ModemStat.obj
 0001:00002274       ReadPDSMPADldData          00103274 f   ModemStat.obj
 0001:000022d8       ReadPDSMPAData             001032d8 f   ModemStat.obj
 0001:000023cc       GetDMMode                  001033cc f   ModemStat.obj
 0001:00002418       GetPTMode                  00103418 f   ModemStat.obj
 0001:00002464       GetActWizUIMask            00103464 f   ModemStat.obj
 0001:000024bc       GetOMADMConfig             001034bc f   ModemStat.obj
 0001:00002514       GetCurrentGSMBandAndList   00103514 f   ModemStat.obj
 0001:000025c0       ??_ECriticalSection@@UAAPAXI@Z 001035c0 f i ModemStat.obj
 0001:000025c0       ??_GCriticalSection@@UAAPAXI@Z 001035c0 f i ModemStat.obj
 0001:000025f0       ??1CModemStatus@@UAA@XZ    001035f0 f   ModemStat.obj
 0001:00002638       ?RilNotifyCallback@@YAXKPBXKK@Z 00103638 f   ModemStat.obj
 0001:0000325c       ??_GCModemStatus@@UAAPAXI@Z 0010425c f i ModemStat.obj
 0001:0000325c       ??_ECModemStatus@@UAAPAXI@Z 0010425c f i ModemStat.obj
 0001:00003280       ?RILInitializeThread@@YAIPAX@Z 00104280 f   ModemStat.obj
 0001:000032f0       ?RILRegister@CModemStatus@@QAAHXZ 001042f0 f   ModemStat.obj
 0001:000033e4       ?Initialize@CModemStatus@@QAAXXZ 001043e4 f   ModemStat.obj
 0001:00003540       ?ClearErrorObjectFunc@@YAXAAUtagErrorInfo@@@Z 00104540 f   ModemStat.obj
 0001:00003578       ?ExecNoParamDevSpecific@@YAHKAAUtagErrorInfo@@@Z 00104578 f   ModemStat.obj
 0001:000036c4       GetUserIdentity            001046c4 f   ModemStat.obj
 0001:00003860       GetRilDebugInfo            00104860 f   ModemStat.obj
 0001:00003a20       GetRilEVDODebugInfo        00104a20 f   ModemStat.obj
 0001:00003a94       GetRilStatus               00104a94 f   ModemStat.obj
 0001:00003b58       GetRilPAParam              00104b58 f   ModemStat.obj
 0001:00003c24       GetRilPDData               00104c24 f   ModemStat.obj
 0001:00003d14       GetRilPDDLDData            00104d14 f   ModemStat.obj
 0001:00003dec       SetEquipmentState          00104dec f   ModemStat.obj
 0001:00003f6c       HangUp                     00104f6c f   ModemStat.obj
 0001:0000407c       Dial                       0010507c f   ModemStat.obj
 0001:000041dc       DialEx                     001051dc f   ModemStat.obj
 0001:000043c0       ModGetPreferredPrivacyMode 001053c0 f   ModemStat.obj
 0001:000044d0       ModGetRoamingMode          001054d0 f   ModemStat.obj
 0001:000045e0       ModSetRoamingMode          001055e0 f   ModemStat.obj
 0001:000046f8       ModSetPreferredPrivacyMode 001056f8 f   ModemStat.obj
 0001:00004810       ModGetLocationStatus       00105810 f   ModemStat.obj
 0001:00004938       ModSetLocationMode         00105938 f   ModemStat.obj
 0001:00004aa8       ModGetRoamStatus           00105aa8 f   ModemStat.obj
 0001:00004bd0       ReadNv                     00105bd0 f   ModemStat.obj
 0001:00004d54       WriteNv                    00105d54 f   ModemStat.obj
 0001:00004ef4       ValidateSpc                00105ef4 f   ModemStat.obj
 0001:000050a4       SetModemPowerState         001060a4 f   ModemStat.obj
 0001:000050dc       GetMDNLengthSupported      001060dc f   ModemStat.obj
 0001:0000515c       SetProvisionInfo           0010615c f   ModemStat.obj
 0001:000053b8       SetSIPNaiPassword          001063b8 f   ModemStat.obj
 0001:0000549c       SaveAkey                   0010649c f   ModemStat.obj
 0001:000055ec       GetVersionInfo             001065ec f   ModemStat.obj
 0001:000058ac       StartDebugMode             001068ac f   ModemStat.obj
 0001:00005a30       StopDebugMode              00106a30 f   ModemStat.obj
 0001:00005bb4       EnableTechHdrNotifications 00106bb4 f   ModemStat.obj
 0001:00005d40       ModGetSysPrefMode          00106d40 f   ModemStat.obj
 0001:00005d4c       ModSetSysPrefMode          00106d4c f   ModemStat.obj
 0001:00005ebc       ModGetHDRHybrPrefMode      00106ebc f   ModemStat.obj
 0001:00005ec8       ModSetHDRHybrPrefMode      00106ec8 f   ModemStat.obj
 0001:00006038       GetIOTALog                 00107038 f   ModemStat.obj
 0001:000061dc       GetIOTALogSize             001071dc f   ModemStat.obj
 0001:0000631c       StartIOTA                  0010731c f   ModemStat.obj
 0001:00006454       StopIOTA                   00107454 f   ModemStat.obj
 0001:0000657c       EnableIOTA                 0010757c f   ModemStat.obj
 0001:000066ec       IsIOTAEnabled              001076ec f   ModemStat.obj
 0001:00006850       GetDsMipList               00107850 f   ModemStat.obj
 0001:00006a1c       GetDsMipProfile            00107a1c f   ModemStat.obj
 0001:00006bd4       SetDsMipProfile            00107bd4 f   ModemStat.obj
 0001:00006d7c       GetByteCounter             00107d7c f   ModemStat.obj
 0001:00006ef0       ReadPDSMPAParam            00107ef0 f   ModemStat.obj
 0001:000070e0       StartLBTrackSession        001080e0 f   ModemStat.obj
 0001:00007290       EndLBTrackSession          00108290 f   ModemStat.obj
 0001:00007418       SetPDSMPAParam             00108418 f   ModemStat.obj
 0001:000075f8       StartPDSMLocNotifstatus    001085f8 f   ModemStat.obj
 0001:00007604       StartPDSMDldNotifstatus    00108604 f   ModemStat.obj
 0001:00007610       StopPDSMLocNotifstatus     00108610 f   ModemStat.obj
 0001:0000761c       StopPDSMDldNotifstatus     0010861c f   ModemStat.obj
 0001:00007628       StartDMMode                00108628 f   ModemStat.obj
 0001:00007798       StopDMMode                 00108798 f   ModemStat.obj
 0001:000077a4       StartPTMode                001087a4 f   ModemStat.obj
 0001:000077b0       StopPTMode                 001087b0 f   ModemStat.obj
 0001:000077bc       GetCallstate               001087bc f   ModemStat.obj
 0001:000078fc       GetProvisionState          001088fc f   ModemStat.obj
 0001:00007a40       InitiateHostBoot           00108a40 f   ModemStat.obj
 0001:00007bb0       RtnReset                   00108bb0 f   ModemStat.obj
 0001:00007d28       SetHdrNaiPassword          00108d28 f   ModemStat.obj
 0001:00007de0       GetHdrNaiPassword          00108de0 f   ModemStat.obj
 0001:00007ee4       GetNAIPWUIDisplayMode      00108ee4 f   ModemStat.obj
 0001:00008068       SendATTunnel               00109068 f   ModemStat.obj
 0001:000082d4       GetGSMInfo                 001092d4 f   ModemStat.obj
 0001:00008408       GetItemnizedUMTSInfo       00109408 f   ModemStat.obj
 0001:000085dc       SelectGSMBand              001095dc f   ModemStat.obj
 0001:0000873c       GetSIPNaiPassword          0010973c f   ModemStat.obj
 0001:0000882c       ?Init@CComCriticalSection@ATL@@QAAJXZ 0010982c f i stdafx.obj
 0001:0000888c       ??1SW_Log@@QAA@XZ          0010988c f   SW_Log.obj
 0001:00008990       ?GetLogFileFromReg@SW_Log@@IAAJPAGAAK@Z 00109990 f   SW_Log.obj
 0001:00008a00       ?GetMaxLogFileReg@SW_Log@@IAAJXZ 00109a00 f   SW_Log.obj
 0001:00008a4c       ?GetCompFilterFromReg@SW_Log@@IAAJAAKK@Z 00109a4c f   SW_Log.obj
 0001:00008ac8       ?GetRetailDebugEnableFromReg@SW_Log@@IAAJPAK@Z 00109ac8 f   SW_Log.obj
 0001:00008b2c       ?GetFilterFromReg@SW_Log@@IAAJAAK@Z 00109b2c f   SW_Log.obj
 0001:00008bd0       ?SetupCOMChannel@SW_Log@@QAAXPAX@Z 00109bd0 f   SW_Log.obj
 0001:00008cd4       ?GetDisplayMemFromReg@SW_Log@@AAAJPAK@Z 00109cd4 f   SW_Log.obj
 0001:00008d80       ?MessageBoxFunction@SW_Log@@KAIPAX@Z 00109d80 f   SW_Log.obj
 0001:00008da4       ?GetModuleFilter@SW_Log@@IAAJPAUHINSTANCE__@@@Z 00109da4 f   SW_Log.obj
 0001:00008e48       ?SWSerialize@SW_Log@@IAAXPAXPBGK@Z 00109e48 f   SW_Log.obj
 0001:000090a0       ?MessageBoxOnSeparateThread@SW_Log@@QAAXPBG@Z 0010a0a0 f   SW_Log.obj
 0001:000090f8       ?Init@SW_Log@@QAAXPAUHINSTANCE__@@@Z 0010a0f8 f   SW_Log.obj
 0001:00009128       ?WriteLog@SW_Log@@QAAXPAGHKPBGPAPAD@Z 0010a128 f   SW_Log.obj
 0001:00009450       ?DisplayLog@SW_Log@@QAAXPBGPAPAD@Z 0010a450 f   SW_Log.obj
 0001:000094b8       ?Run@SW_Log@@IAAXXZ        0010a4b8 f   SW_Log.obj
 0001:00009678       ?LogThreadFunc@SW_Log@@CAXPAX@Z 0010a678 f   SW_Log.obj
 0001:0000967c       ?InitObject@SW_Log@@IAAXXZ 0010a67c f   SW_Log.obj
 0001:0000981c       ?InitLog@@YAXPAUHINSTANCE__@@@Z 0010a81c f   SW_Log_Include.obj
 0001:0000982c       ?WriteLog@@YAXPAVSW_Log@@KPBGPAPAD@Z 0010a82c f   SW_Log_Include.obj
 0001:00009864       ?WriteLog@@YAXPAVSW_Log@@KPBGZZ 0010a864 f   SW_Log_Include.obj
 0001:000098b0       ?WriteLog@@YAXKPBGZZ       0010a8b0 f   SW_Log_Include.obj
 0001:00009904       ?LogV@@YAXPBGZZ            0010a904 f   SW_Log_Include.obj
 0001:00009958       ?LogC@@YAXPBGZZ            0010a958 f   SW_Log_Include.obj
 0001:000099ac       ?LogW@@YAXPBGZZ            0010a9ac f   SW_Log_Include.obj
 0001:00009a00       ?LogWindowText@@YAXPBGZZ   0010aa00 f   SW_Log_Include.obj
 0001:00009a38       ?LogStoreFileLine@@YAXPAGH@Z 0010aa38 f   SW_Log_Include.obj
 0001:00009a5c       ?GetAvailStoreMem@@YAKXZ   0010aa5c f   SW_Log_Include.obj
 0001:00009a78       ?GetAvailMem@@YAKXZ        0010aa78 f   SW_Log_Include.obj
 0001:00009a9c       ?GetMemUsed@@YAKXZ         0010aa9c f   SW_Log_Include.obj
 0001:00009ac8       ?TBD_Assert@@YA_N_NQBG1H@Z 0010aac8 f   SW_Log_Include.obj
 0001:00009b04       ?TBD_Output@@YAXW4TBD_CLASS_TYPE@@W4TBD_OUTPUT_LEVEL@@QBGZZ 0010ab04 f   SW_Log_Include.obj
 0001:00009b68       ?DisplayRawData@@YAXIPAEHPBG@Z 0010ab68 f   SW_Log_Include.obj
 0001:00009d60       ?WriteLog@@YAXPAVSW_Log@@PBGZZ 0010ad60 f   SW_Log_Include.obj
 0001:00009dac       ?WriteLog@@YAXPBGZZ        0010adac f   SW_Log_Include.obj
 0001:00009e00       ?GetAvailProgramMem@@YAKXZ 0010ae00 f   SW_Log_Include.obj
 0001:00009e34       ?DeleteSubKey@SW_RegistryKey@@IAAJPBG@Z 0010ae34 f   SW_Registrykey.obj
 0001:00009e3c       ?InitObject@SW_RegistryKey@@MAAXXZ 0010ae3c f   SW_Registrykey.obj
 0001:00009e4c       ?CreateKey@SW_RegistryKey@@UAAJPBGKPAK@Z 0010ae4c f   SW_Registrykey.obj
 0001:00009e80       ?OpenKey@SW_RegistryKey@@UAAJPBGK@Z 0010ae80 f   SW_Registrykey.obj
 0001:00009eac       ?OpenKey@SW_RegistryKey@@UAAJPAUHKEY__@@PBGK@Z 0010aeac f   SW_Registrykey.obj
 0001:00009ee0       ?CloseKey@SW_RegistryKey@@UAAJXZ 0010aee0 f   SW_Registrykey.obj
 0001:00009f1c       ?QueryValue@SW_RegistryKey@@UAAJPBGPAPAG@Z 0010af1c f   SW_Registrykey.obj
 0001:0000a030       ?QueryValue@SW_RegistryKey@@UAAJPBGPAK@Z 0010b030 f   SW_Registrykey.obj
 0001:0000a0d0       ?QueryValue@SW_RegistryKey@@UAAJPBGPAPAEPAK@Z 0010b0d0 f   SW_Registrykey.obj
 0001:0000a1c0       ?SetValue@SW_RegistryKey@@UAAJPBG0@Z 0010b1c0 f   SW_Registrykey.obj
 0001:0000a208       ?SetValue@SW_RegistryKey@@UAAJPBGK@Z 0010b208 f   SW_Registrykey.obj
 0001:0000a240       ?SetValue@SW_RegistryKey@@UAAJPBGQAEK@Z 0010b240 f   SW_Registrykey.obj
 0001:0000a270       ?EnumKey@SW_RegistryKey@@IAAJAAKPAG@Z 0010b270 f   SW_Registrykey.obj
 0001:0000a2b8       ??0SW_RegistryKey@@QAA@XZ  0010b2b8 f   SW_Registrykey.obj
 0001:0000a2d4       ??0SW_RegistryKey@@QAA@PAUHKEY__@@@Z 0010b2d4 f   SW_Registrykey.obj
 0001:0000a2f0       ??1SW_RegistryKey@@QAA@XZ  0010b2f0 f   SW_Registrykey.obj
 0001:0000a334       ?CreateKey@SW_RegistryKey@@UAAJPAUHKEY__@@PBGKPAK@Z 0010b334 f   SW_Registrykey.obj
 0001:0000a484       ?Duplicate@SW_RegistryKey@@QAAHAAV1@@Z 0010b484 f   SW_Registrykey.obj
 0001:0000a744       ?GetRegValue@@YAJPAUHKEY__@@PBG1AAK@Z 0010b744 f   SW_Registrykey.obj
 0001:0000a850       ?GetRegValue@@YAJPAUHKEY__@@PBG1PAGPAK@Z 0010b850 f   SW_Registrykey.obj
 0001:0000a980       ?GetRegValue@@YAJPAUHKEY__@@PBG1PAEPAK@Z 0010b980 f   SW_Registrykey.obj
 0001:0000aa90       ?SetRegValue@@YAJPAUHKEY__@@PBG11@Z 0010ba90 f   SW_Registrykey.obj
 0001:0000ab58       ?SetRegValue@@YAJPAUHKEY__@@PBG1QAEK@Z 0010bb58 f   SW_Registrykey.obj
 0001:0000ac30       ?SetRegValue@@YAJPAUHKEY__@@PBG1K@Z 0010bc30 f   SW_Registrykey.obj
 0001:0000acf8       ?SWAI_GetRegValue@@YAJPAUHKEY__@@PBG1AAK@Z 0010bcf8 f   SW_Registrykey.obj
 0001:0000ae5c       ?SWAI_GetRegValue@@YAJPAUHKEY__@@PBG1PAGPAK@Z 0010be5c f   SW_Registrykey.obj
 0001:0000b028       ?SWAI_GetRegValue@@YAJPAUHKEY__@@PBG1PAEPAK@Z 0010c028 f   SW_Registrykey.obj
 0001:0000b1dc       ?SWAI_SetRegValue@@YAJPAUHKEY__@@PBG11@Z 0010c1dc f   SW_Registrykey.obj
 0001:0000b318       ?SWAI_SetRegValue@@YAJPAUHKEY__@@PBG1QAEK@Z 0010c318 f   SW_Registrykey.obj
 0001:0000b45c       ?SWAI_SetRegValue@@YAJPAUHKEY__@@PBG1K@Z 0010c45c f   SW_Registrykey.obj
 0001:0000b598       ?CopyRegKey@@YAJPAUHKEY__@@PBG11H@Z 0010c598 f   SW_Registrykey.obj
 0001:0000b864       ?RecurseDeleteKey@SW_RegistryKey@@QAAJPBG@Z 0010c864 f   SW_Registrykey.obj
 0001:0000b9ac       ?DeleteRegKey@@YAJPAUHKEY__@@PBG1H@Z 0010c9ac f   SW_Registrykey.obj
 0001:0000bbbc       ?RenameRegKey@@YAJPAUHKEY__@@PBG11H@Z 0010cbbc f   SW_Registrykey.obj
 0001:0000bec0       ?GetVerInfo@@YAPAGPAUHINSTANCE__@@@Z 0010cec0 f   Utilities.obj
 0001:0000bfc0       ?GetOSVersioninfo@@YAXXZ   0010cfc0 f   Utilities.obj
 0001:0000c00c       ?GetDataPortDetails@@YAHPAGAAK@Z 0010d00c f   Utilities.obj
 0001:0000c0ec       ?GetCarrierIndex@@YAKXZ    0010d0ec f   Utilities.obj
 0001:0000c278       ?SetAutoUpdateTime@@YAXH@Z 0010d278 f   Utilities.obj
 0001:0000c294       ?SetAutoUpdateTimeUI@@YAXK@Z 0010d294 f   Utilities.obj
 0001:0000c2b0       ?SetCallGuardReg@@YAXK@Z   0010d2b0 f   Utilities.obj
 0001:0000c2cc       ?GetActWizDisabled@@YAKXZ  0010d2cc f   Utilities.obj
 0001:0000c304       ?SetActWizDisabled@@YAXK@Z 0010d304 f   Utilities.obj
 0001:0000c320       ?GetMdnLen@@YAHAAK@Z       0010d320 f   Utilities.obj
 0001:0000c378       ?IsConsumerProduct@@YAHXZ  0010d378 f   Utilities.obj
 0001:0000c3c4       ?GetLogoTestReg@@YAKXZ     0010d3c4 f   Utilities.obj
 0001:0000c408       ?EnableCarrierLogo@@YAXH@Z 0010d408 f   Utilities.obj
 0001:0000c484       ?EncodeMCC1112@@YAHPBG_N@Z 0010d484 f   Utilities.obj
 0001:0000c4dc       ?EncodePhoneNumber@@YA_NPAGPAK@Z 0010d4dc f   Utilities.obj
 0001:0000c6c8       ?DecodeMCC1112@@YAHH_N@Z   0010d6c8 f   Utilities.obj
 0001:0000c78c       ?SW_AtoT@@YAPAGPAGPADK@Z   0010d78c f   Utilities.obj
 0001:0000c7b0       ?SW_TtoA@@YAPADPADPAGK@Z   0010d7b0 f   Utilities.obj
 0001:0000c7d0       ?GetProductFeatures@@YAHAAK@Z 0010d7d0 f   Utilities.obj
 0001:0000ca0c       ?InWideMode@@YAHXZ         0010da0c f   Utilities.obj
 0001:0000ca38       ?SetLimitText@@YAJPAUHWND__@@H@Z 0010da38 f   Utilities.obj
 0001:0000ca48       ?GetResolution@@YAHXZ      0010da48 f   Utilities.obj
 0001:0000ca8c       ?SetConnectionProfile@@YAJXZ 0010da8c f   Utilities.obj
 0001:0000d094       ?EnableLocationReg@@YAJXZ  0010e094 f   Utilities.obj
 0001:0000d1c8       ?SetLocationResourceBaseID@@YAJK@Z 0010e1c8 f   Utilities.obj
 0001:0000d3f8       ?SetSpecialNumber@@YAJPAG@Z 0010e3f8 f   Utilities.obj
 0001:0000d490       ?GetSpecialNumber@@YAJPAG@Z 0010e490 f   Utilities.obj
 0001:0000d550       ?SetNormalCursor@@YAXXZ    0010e550 f   Utilities.obj
 0001:0000d568       ?SetWaitCursor@@YAXXZ      0010e568 f   Utilities.obj
 0001:0000d588       ?ConvertPrefMode@@YAH_NH@Z 0010e588 f   Utilities.obj
 0001:0000d638       ?BtoH@@YAED@Z              0010e638 f   Utilities.obj
 0001:0000d688       ?TtoTH@@YAXPAG0H@Z         0010e688 f   Utilities.obj
 0001:0000d748       ?THtoT@@YAXPAG0H@Z         0010e748 f   Utilities.obj
 0001:0000d83c       ?LocalToUTCTime@@YAHPAU_SYSTEMTIME@@0@Z 0010e83c f   Utilities.obj
 0001:0000d89c       ?DWORD2IP@@YAPBGK@Z        0010e89c f   Utilities.obj
 0001:0000d918       ?ChangeCarrierIndex@@YAJKK@Z 0010e918 f   Utilities.obj
 0001:0000dba4       ?GetAutoUpdateTimeUI@@YAKXZ 0010eba4 f   Utilities.obj
 0001:0000dbf8       ?GetAutoUpdateTime@@YAKXZ  0010ebf8 f   Utilities.obj
 0001:0000dc4c       ?GetCallGuardReg@@YAKXZ    0010ec4c f   Utilities.obj
 0001:0000dc9c       ?DecodeAreaCode@@YA_NPAGG@Z 0010ec9c f   Utilities.obj
 0001:0000dd60       ?DecodePhoneNumber@@YA_NPAGK@Z 0010ed60 f   Utilities.obj
 0001:0000deb0       ?RelayoutDialog@@YAHPAUHINSTANCE__@@PAUHWND__@@PBG@Z 0010eeb0 f   Utilities.obj
 0001:0000e138       ?IP2DWORD@@YAKPBG@Z        0010f138 f   Utilities.obj
 0001:0000e2bc       memcpy                     0010f2bc f   coredll:COREDLL.dll
 0001:0000e2cc       ??3@YAXPAX@Z               0010f2cc f   coredll:COREDLL.dll
 0001:0000e2dc       GetFileVersionInfoW        0010f2dc f   coredll:COREDLL.dll
 0001:0000e2ec       ??2@YAPAXI@Z               0010f2ec f   coredll:COREDLL.dll
 0001:0000e2fc       GetFileVersionInfoSizeW    0010f2fc f   coredll:COREDLL.dll
 0001:0000e30c       wcscpy                     0010f30c f   coredll:COREDLL.dll
 0001:0000e31c       OutputDebugStringW         0010f31c f   coredll:COREDLL.dll
 0001:0000e32c       swprintf                   0010f32c f   coredll:COREDLL.dll
 0001:0000e33c       VerQueryValueW             0010f33c f   coredll:COREDLL.dll
 0001:0000e34c       wcscat                     0010f34c f   coredll:COREDLL.dll
 0001:0000e35c       GetModuleFileNameW         0010f35c f   coredll:COREDLL.dll
 0001:0000e36c       EventModify                0010f36c f   coredll:COREDLL.dll
 0001:0000e37c       InitializeCriticalSection  0010f37c f   coredll:COREDLL.dll
 0001:0000e38c       DeleteCriticalSection      0010f38c f   coredll:COREDLL.dll
 0001:0000e39c       EnterCriticalSection       0010f39c f   coredll:COREDLL.dll
 0001:0000e3ac       LeaveCriticalSection       0010f3ac f   coredll:COREDLL.dll
 0001:0000e3bc       RegisterWindowMessageW     0010f3bc f   coredll:COREDLL.dll
 0001:0000e3cc       CreateEventW               0010f3cc f   coredll:COREDLL.dll
 0001:0000e3dc       wsprintfW                  0010f3dc f   coredll:COREDLL.dll
 0001:0000e3ec       WaitForSingleObject        0010f3ec f   coredll:COREDLL.dll
 0001:0000e3fc       memset                     0010f3fc f   coredll:COREDLL.dll
 0001:0000e40c       PostMessageW               0010f40c f   coredll:COREDLL.dll
 0001:0000e41c       CloseHandle                0010f41c f   coredll:COREDLL.dll
 0001:0000e42c       CreateThread               0010f42c f   coredll:COREDLL.dll
 0001:0000e43c       wcslen                     0010f43c f   coredll:COREDLL.dll
 0001:0000e44c       strcpy                     0010f44c f   coredll:COREDLL.dll
 0001:0000e45c       wcsncpy                    0010f45c f   coredll:COREDLL.dll
 0001:0000e46c       strlen                     0010f46c f   coredll:COREDLL.dll
 0001:0000e47c       __C_specific_handler       0010f47c f   coredll:COREDLL.dll
 0001:0000e48c       free                       0010f48c f   coredll:COREDLL.dll
 0001:0000e49c       CloseMsgQueue              0010f49c f   coredll:COREDLL.dll
 0001:0000e4ac       TerminateThread            0010f4ac f   coredll:COREDLL.dll
 0001:0000e4bc       WriteMsgQueue              0010f4bc f   coredll:COREDLL.dll
 0001:0000e4cc       PurgeComm                  0010f4cc f   coredll:COREDLL.dll
 0001:0000e4dc       SetCommMask                0010f4dc f   coredll:COREDLL.dll
 0001:0000e4ec       SetCommTimeouts            0010f4ec f   coredll:COREDLL.dll
 0001:0000e4fc       SetCommState               0010f4fc f   coredll:COREDLL.dll
 0001:0000e50c       GetCommState               0010f50c f   coredll:COREDLL.dll
 0001:0000e51c       MessageBoxW                0010f51c f   coredll:COREDLL.dll
 0001:0000e52c       wcsstr                     0010f52c f   coredll:COREDLL.dll
 0001:0000e53c       _wcslwr                    0010f53c f   coredll:COREDLL.dll
 0001:0000e54c       DeleteFileW                0010f54c f   coredll:COREDLL.dll
 0001:0000e55c       FlushFileBuffers           0010f55c f   coredll:COREDLL.dll
 0001:0000e56c       WriteFile                  0010f56c f   coredll:COREDLL.dll
 0001:0000e57c       GetLastError               0010f57c f   coredll:COREDLL.dll
 0001:0000e58c       CreateFileW                0010f58c f   coredll:COREDLL.dll
 0001:0000e59c       CopyFileW                  0010f59c f   coredll:COREDLL.dll
 0001:0000e5ac       GetFileSize                0010f5ac f   coredll:COREDLL.dll
 0001:0000e5bc       Sleep                      0010f5bc f   coredll:COREDLL.dll
 0001:0000e5cc       NKDbgPrintfW               0010f5cc f   coredll:COREDLL.dll
 0001:0000e5dc       GetLocalTime               0010f5dc f   coredll:COREDLL.dll
 0001:0000e5ec       vswprintf                  0010f5ec f   coredll:COREDLL.dll
 0001:0000e5fc       wcscmp                     0010f5fc f   coredll:COREDLL.dll
 0001:0000e60c       ReadMsgQueue               0010f60c f   coredll:COREDLL.dll
 0001:0000e61c       CreateMsgQueue             0010f61c f   coredll:COREDLL.dll
 0001:0000e62c       SetFilePointer             0010f62c f   coredll:COREDLL.dll
 0001:0000e63c       ReleaseMutex               0010f63c f   coredll:COREDLL.dll
 0001:0000e64c       CreateMutexW               0010f64c f   coredll:COREDLL.dll
 0001:0000e65c       GetStoreInformation        0010f65c f   coredll:COREDLL.dll
 0001:0000e66c       GlobalMemoryStatus         0010f66c f   coredll:COREDLL.dll
 0001:0000e67c       rand                       0010f67c f   coredll:COREDLL.dll
 0001:0000e68c       RegDeleteKeyW              0010f68c f   coredll:COREDLL.dll
 0001:0000e69c       RegOpenKeyExW              0010f69c f   coredll:COREDLL.dll
 0001:0000e6ac       RegCloseKey                0010f6ac f   coredll:COREDLL.dll
 0001:0000e6bc       RegQueryValueExW           0010f6bc f   coredll:COREDLL.dll
 0001:0000e6cc       RegSetValueExW             0010f6cc f   coredll:COREDLL.dll
 0001:0000e6dc       RegEnumKeyExW              0010f6dc f   coredll:COREDLL.dll
 0001:0000e6ec       wcschr                     0010f6ec f   coredll:COREDLL.dll
 0001:0000e6fc       RegCreateKeyExW            0010f6fc f   coredll:COREDLL.dll
 0001:0000e70c       RegEnumValueW              0010f70c f   coredll:COREDLL.dll
 0001:0000e71c       GetVersionExW              0010f71c f   coredll:COREDLL.dll
 0001:0000e72c       _wcsicmp                   0010f72c f   coredll:COREDLL.dll
 0001:0000e73c       _wtol                      0010f73c f   coredll:COREDLL.dll
 0001:0000e74c       mbstowcs                   0010f74c f   coredll:COREDLL.dll
 0001:0000e75c       wcstombs                   0010f75c f   coredll:COREDLL.dll
 0001:0000e76c       SetDlgItemTextW            0010f76c f   coredll:COREDLL.dll
 0001:0000e77c       DeleteObject               0010f77c f   coredll:COREDLL.dll
 0001:0000e78c       LoadBitmapW                0010f78c f   coredll:COREDLL.dll
 0001:0000e79c       DestroyIcon                0010f79c f   coredll:COREDLL.dll
 0001:0000e7ac       LoadIconW                  0010f7ac f   coredll:COREDLL.dll
 0001:0000e7bc       SendDlgItemMessageW        0010f7bc f   coredll:COREDLL.dll
 0001:0000e7cc       GetSystemMetrics           0010f7cc f   coredll:COREDLL.dll
 0001:0000e7dc       SendMessageW               0010f7dc f   coredll:COREDLL.dll
 0001:0000e7ec       FreeLibrary                0010f7ec f   coredll:COREDLL.dll
 0001:0000e7fc       GetProcAddressW            0010f7fc f   coredll:COREDLL.dll
 0001:0000e80c       LoadLibraryW               0010f80c f   coredll:COREDLL.dll
 0001:0000e81c       RegDeleteValueW            0010f81c f   coredll:COREDLL.dll
 0001:0000e82c       SetCursor                  0010f82c f   coredll:COREDLL.dll
 0001:0000e83c       LoadCursorW                0010f83c f   coredll:COREDLL.dll
 0001:0000e84c       FileTimeToSystemTime       0010f84c f   coredll:COREDLL.dll
 0001:0000e85c       LocalFileTimeToFileTime    0010f85c f   coredll:COREDLL.dll
 0001:0000e86c       SystemTimeToFileTime       0010f86c f   coredll:COREDLL.dll
 0001:0000e87c       EndDeferWindowPos          0010f87c f   coredll:COREDLL.dll
 0001:0000e88c       DeferWindowPos             0010f88c f   coredll:COREDLL.dll
 0001:0000e89c       MapDialogRect              0010f89c f   coredll:COREDLL.dll
 0001:0000e8ac       GetDlgItem                 0010f8ac f   coredll:COREDLL.dll
 0001:0000e8bc       BeginDeferWindowPos        0010f8bc f   coredll:COREDLL.dll
 0001:0000e8cc       LoadResource               0010f8cc f   coredll:COREDLL.dll
 0001:0000e8dc       FindResourceW              0010f8dc f   coredll:COREDLL.dll
 0001:0000e8ec       RIL_Deinitialize           0010f8ec f   ril:ril.dll
 0001:0000e8fc       RIL_DevSpecific            0010f8fc f   ril:ril.dll
 0001:0000e90c       RIL_GetEquipmentState      0010f90c f   ril:ril.dll
 0001:0000e91c       RIL_GetRegistrationStatus  0010f91c f   ril:ril.dll
 0001:0000e92c       RIL_GetCurrentSystemType   0010f92c f   ril:ril.dll
 0001:0000e93c       RIL_GetCallList            0010f93c f   ril:ril.dll
 0001:0000e94c       RIL_Initialize             0010f94c f   ril:ril.dll
 0001:0000e95c       RIL_GetUserIdentity        0010f95c f   ril:ril.dll
 0001:0000e96c       RIL_SetEquipmentState      0010f96c f   ril:ril.dll
 0001:0000e97c       RIL_Hangup                 0010f97c f   ril:ril.dll
 0001:0000e98c       RIL_Dial                   0010f98c f   ril:ril.dll
 0001:0000e99c       RIL_GetPreferredPrivacyMode 0010f99c f   ril:ril.dll
 0001:0000e9ac       RIL_GetRoamingMode         0010f9ac f   ril:ril.dll
 0001:0000e9bc       RIL_SetRoamingMode         0010f9bc f   ril:ril.dll
 0001:0000e9cc       RIL_SetPreferredPrivacyMode 0010f9cc f   ril:ril.dll
 0001:0000e9dc       RIL_SendAKey               0010f9dc f   ril:ril.dll
 0001:0000e9ec       RIL_GetPacketByteCount     0010f9ec f   ril:ril.dll
 0001:0000e9fc       ntohl                      0010f9fc f   ws2:WS2.dll
 0001:0000ea0c       _DllMainCRTStartup         0010fa0c f   corelibc:pegdmain.obj
 0001:0000eaa4       __security_check_cookie    0010faa4     corelibc:armsecgs.obj
 0001:0000eab8       __gsfailure                0010fab8     corelibc:armsecgs.obj
 0001:0000eafc       _onexit                    0010fafc f   corelibc:onexit.obj
 0001:0000eba8       atexit                     0010fba8 f   corelibc:onexit.obj
 0001:0000ebc8       _cinit                     0010fbc8 f   corelibc:crt0dat.obj
 0001:0000ed38       _cexit                     0010fd38 f   corelibc:crt0dat.obj
 0001:0000ed54       DllMain                    0010fd54 f   corelibc:dllmain.obj
 0001:0000ed6c       __security_init_cookie     0010fd6c f   corelibc:seccinit.obj
 0001:0000edbc       AtlRawDllMain              0010fdbc f   atls:atlbase.obj
 0001:0000ee54       ?RemoveAll@?$CSimpleArray@PAUHINSTANCE__@@V?$CSimpleArrayEqualHelper@PAUHINSTANCE__@@@ATL@@@ATL@@QAAXXZ 0010fe54 f i atls:atlbase.obj
 0001:0000ee90       ??0_ATL_BASE_MODULE70@ATL@@QAA@XZ 0010fe90 f i atls:atlbase.obj
 0001:0000eed4       ??1CAtlBaseModule@ATL@@QAA@XZ 0010fed4 f   atls:atlbase.obj
 0001:0000ef0c       ??0CAtlBaseModule@ATL@@QAA@XZ 0010ff0c f   atls:atlbase.obj
 0001:0000efa8       __GSHandlerCheckCommon     0010ffa8 f   LIBCMT:gshandler.obj
 0001:0000eff0       __GSHandlerCheck           0010fff0 f   LIBCMT:gshandler.obj
 0001:0000f028       __FrameUnwindToState       00110028 f   LIBCMT:frame_ce.obj
 0001:0000f3a0       ?_DestructExceptionObject@@YAXPAUEHExceptionRecord@@E@Z 001103a0 f   LIBCMT:frame_ce.obj
 0001:0000f40c       ?_OffsetToAddress@@YAPAXHPAKK@Z 0011040c f   LIBCMT:frame_ce.obj
 0001:0000f458       ?FindFrameInfo@@YAPAU_FrameInfo@@PAK@Z 00110458 f   LIBCMT:frame_ce.obj
 0001:0000f498       ?FindCatchFrameInfo@@YAPAU_FrameInfo@@PAK@Z 00110498 f   LIBCMT:frame_ce.obj
 0001:0000f4d8       ?_GetRangeOfTrysToCheck@@YAPBU_s_TryBlockMapEntry@@PBU_s_FuncInfo@@HHPAI1@Z 001104d8 f   LIBCMT:frame_ce.obj
 0001:0000fee4       __InternalCxxFrameHandler  00110ee4 f   LIBCMT:frame_ce.obj
 0001:0001003c       __CxxFrameHandler3         0011103c f   LIBCMT:frame_ce.obj
 0001:00010074       __GSHandlerCheck_EH        00111074 f   LIBCMT:gshandlereh.obj
 0001:00010108       GetCRTStorage              00111108 f   LIBCMT:corecrt.obj
 0001:000101d4       _CallSettingFrame          001111d4     LIBCMT:handlers_arm.obj
 0001:00010218       ?FindFrameForUnwind@@YAPAKPAKPBU_s_FuncInfo@@@Z 00111218 f   LIBCMT:mdframe_arm.obj
 0001:00010260       ?FindCatchFrame@@YAPAKPAKK@Z 00111260 f   LIBCMT:mdframe_arm.obj
 0001:000102ac       ?AdjustFrameForCatch@@YAPAKPAKPBU_s_FuncInfo@@@Z 001112ac f   LIBCMT:mdframe_arm.obj
 0001:000102e4       ?GetCurrentState@@YAHPAKPAU_DISPATCHER_CONTEXT@@PBU_s_FuncInfo@@@Z 001112e4 f   LIBCMT:ehstate_arm_mips.obj
 0001:00010340       __report_gsfailure         00111340 f   coredll:COREDLL.dll
 0001:00010350       LocalReAlloc               00111350 f   coredll:COREDLL.dll
 0001:00010360       LocalAlloc                 00111360 f   coredll:COREDLL.dll
 0001:00010370       LocalSize                  00111370 f   coredll:COREDLL.dll
 0001:00010380       LocalFree                  00111380 f   coredll:COREDLL.dll
 0001:00010390       DisableThreadLibraryCalls  00111390 f   coredll:COREDLL.dll
 0001:000103a0       __security_gen_cookie      001113a0 f   coredll:COREDLL.dll
 0001:000103b0       GetModuleHandleW           001113b0 f   coredll:COREDLL.dll
 0001:000103c0       strcmp                     001113c0 f   coredll:COREDLL.dll
 0001:000103d0       ?terminate@std@@YAXXZ      001113d0 f   coredll:COREDLL.dll
 0001:000103e0       memmove                    001113e0 f   coredll:COREDLL.dll
 0001:000103f0       TlsCall                    001113f0 f   coredll:COREDLL.dll
 0001:00010400       TlsSetValue                00111400 f   coredll:COREDLL.dll
 0001:00010410       TlsGetValue                00111410 f   coredll:COREDLL.dll
 0001:00010420       InterlockedCompareExchange 00111420 f   coredll:COREDLL.dll
 0002:00000000       ??_C@_1DE@EMJBEPGN@?$AA?2?$AAS?$AAt?$AAr?$AAi?$AAn?$AAg?$AAF?$AAi?$AAl?$AAe?$AAI?$AAn?$AAf?$AAo?$AA?2?$AA0?$AA4?$AA0?$AA9?$AA0?$AA4?$AAB?$AA0?$AA?2?$AA?$AA@ 00112000     CVERINFO.obj
 0002:00000038       ??_C@_1EA@GNKGCCEH@?$AA?4?$AA?4?$AA?2?$AA?4?$AA?4?$AA?2?$AA?4?$AA?4?$AA?2?$AA?4?$AA?4?$AA?2?$AAC?$AAo?$AAm?$AAm?$AAo?$AAn?$AA?2?$AAC?$AAV?$AAE?$AAR?$AAI?$AAN?$AAF?$AAO?$AA?4?$AAC?$AAP?$AAP?$AA?$AA@ 00112038     CVERINFO.obj
 0002:00000078       ??_C@_1GA@LFAMMLJO@?$AAG?$AAe?$AAt?$AAF?$AAi?$AAl?$AAe?$AAV?$AAe?$AAr?$AAs?$AAi?$AAo?$AAn?$AAI?$AAn?$AAf?$AAo?$AAS?$AAi?$AAz?$AAe?$AA?5?$AAr?$AAe?$AAt?$AAu?$AAr?$AAn?$AAs?$AA?5?$AAs@ 00112078     CVERINFO.obj
 0002:000000d8       ??_C@_1DM@IOFBAEKC@?$AA?$CF?$AAs?$AA?5?$AAh?$AAa?$AAs?$AA?5?$AAn?$AAo?$AA?5?$AAv?$AAe?$AAr?$AAs?$AAi?$AAo?$AAn?$AA?5?$AAr?$AAe?$AAs?$AAs?$AAo?$AAu?$AAr?$AAc?$AAe?$AA?$AN?$AA?6?$AA?$AA@ 001120d8     CVERINFO.obj
 0002:00000114       ??_C@_1BI@CJGIOPAN@?$AAP?$AAr?$AAo?$AAd?$AAu?$AAc?$AAt?$AAN?$AAa?$AAm?$AAe?$AA?$AA@ 00112114     CVERINFO.obj
 0002:0000012c       ??_C@_1BI@HCCAONKE@?$AAF?$AAi?$AAl?$AAe?$AAV?$AAe?$AAr?$AAs?$AAi?$AAo?$AAn?$AA?$AA@ 0011212c     CVERINFO.obj
 0002:00000144       ??_C@_1BO@OKEPMKJE@?$AAP?$AAr?$AAo?$AAd?$AAu?$AAc?$AAt?$AAV?$AAe?$AAr?$AAs?$AAi?$AAo?$AAn?$AA?$AA@ 00112144     CVERINFO.obj
 0002:00000164       ??_7SW_RegistryKey@@6B@    00112164     ModemStat.obj
 0002:00000198       ??_7CriticalSection@@6B@   00112198     ModemStat.obj
 0002:0000019c       ??_C@_1CG@POBHOMMK@?$AAR?$AAI?$AAL?$AA_?$AAS?$AAT?$AAA?$AAT?$AAU?$AAS?$AA_?$AAC?$AAH?$AAA?$AAN?$AAG?$AAE?$AAD?$AA?$AA@ 0011219c     ModemStat.obj
 0002:000001c4       ??_C@_1BO@NKICKCPO@?$AAR?$AAI?$AAL?$AA_?$AAD?$AAB?$AAG?$AA_?$AAN?$AAO?$AAT?$AAI?$AAF?$AAY?$AA?$AA@ 001121c4     ModemStat.obj
 0002:000001e4       ??_C@_1CG@HIPGCNFB@?$AAR?$AAI?$AAL?$AA_?$AAT?$AAE?$AAC?$AAH?$AAH?$AAD?$AAR?$AA_?$AAN?$AAO?$AAT?$AAI?$AAF?$AAY?$AA?$AA@ 001121e4     ModemStat.obj
 0002:0000020c       ??_C@_1DA@MPHILDIE@?$AAR?$AAI?$AAL?$AA_?$AAI?$AAO?$AAT?$AAA?$AA_?$AAS?$AAT?$AAA?$AAT?$AAU?$AAS?$AA_?$AAC?$AAH?$AAA?$AAN?$AAG?$AAE?$AAD?$AA?$AA@ 0011220c     ModemStat.obj
 0002:0000023c       ??_C@_1CC@BEOCDLIL@?$AAR?$AAI?$AAL?$AA_?$AAI?$AAO?$AAT?$AAA?$AA_?$AAW?$AAA?$AAP?$AA_?$AAU?$AAR?$AAI?$AA?$AA@ 0011223c     ModemStat.obj
 0002:00000260       ??_C@_1CC@POEPKLA@?$AAR?$AAI?$AAL?$AA_?$AAP?$AAD?$AAS?$AAM?$AA_?$AAP?$AAD?$AA_?$AAD?$AAA?$AAT?$AAA?$AA?$AA@ 00112260     ModemStat.obj
 0002:00000284       ??_C@_1CC@DHEBFOCI@?$AAR?$AAI?$AAL?$AA_?$AAP?$AAD?$AAS?$AAM?$AA_?$AAP?$AAD?$AA_?$AAD?$AAO?$AAN?$AAE?$AA?$AA@ 00112284     ModemStat.obj
 0002:000002a8       ??_C@_1CA@IJMMNJBM@?$AAR?$AAI?$AAL?$AA_?$AAP?$AAD?$AAS?$AAM?$AA_?$AAP?$AAD?$AA_?$AAE?$AAN?$AAD?$AA?$AA@ 001122a8     ModemStat.obj
 0002:000002c8       ??_C@_1CE@DKNHCEGP@?$AAR?$AAI?$AAL?$AA_?$AAP?$AAD?$AAS?$AAM?$AA_?$AAP?$AAD?$AA_?$AAB?$AAE?$AAG?$AAI?$AAN?$AA?$AA@ 001122c8     ModemStat.obj
 0002:000002ec       ??_C@_1DG@ENNLKGLF@?$AAR?$AAI?$AAL?$AA_?$AAP?$AAD?$AAS?$AAM?$AA_?$AAP?$AAD?$AA_?$AAU?$AAP?$AAD?$AAA?$AAT?$AAE?$AA_?$AAF?$AAA?$AAI?$AAL?$AAU?$AAR?$AAE?$AA?$AA@ 001122ec     ModemStat.obj
 0002:00000324       ??_C@_1CK@FFHNCNLC@?$AAR?$AAI?$AAL?$AA_?$AAP?$AAD?$AAS?$AAM?$AA_?$AAP?$AAD?$AA_?$AAD?$AAL?$AAD?$AA_?$AAD?$AAA?$AAT?$AAA?$AA?$AA@ 00112324     ModemStat.obj
 0002:00000350       ??_C@_1CK@GNNIIJCK@?$AAR?$AAI?$AAL?$AA_?$AAP?$AAD?$AAS?$AAM?$AA_?$AAP?$AAD?$AA_?$AAD?$AAL?$AAD?$AA_?$AAD?$AAO?$AAN?$AAE?$AA?$AA@ 00112350     ModemStat.obj
 0002:0000037c       ??_C@_1CI@IINDIONI@?$AAR?$AAI?$AAL?$AA_?$AAP?$AAD?$AAS?$AAM?$AA_?$AAP?$AAD?$AA_?$AAD?$AAL?$AAD?$AA_?$AAE?$AAN?$AAD?$AA?$AA@ 0011237c     ModemStat.obj
 0002:000003a4       ??_C@_1CM@BAFGFLAD@?$AAR?$AAI?$AAL?$AA_?$AAP?$AAD?$AAS?$AAM?$AA_?$AAP?$AAD?$AA_?$AAD?$AAL?$AAD?$AA_?$AAB?$AAE?$AAG?$AAI?$AAN?$AA?$AA@ 001123a4     ModemStat.obj
 0002:000003d0       ??_C@_1CE@GDPLDIKM@?$AAR?$AAI?$AAL?$AA_?$AAP?$AAD?$AAS?$AAM?$AA_?$AAP?$AAA?$AA_?$AAP?$AAA?$AAR?$AAA?$AAM?$AA?$AA@ 001123d0     ModemStat.obj
 0002:000003f4       ??_C@_1CE@ILHCKNGC@?$AAR?$AAI?$AAL?$AA_?$AAC?$AAA?$AAL?$AAL?$AA_?$AAB?$AAY?$AAT?$AAE?$AA_?$AAC?$AAT?$AAR?$AA?$AA@ 001123f4     ModemStat.obj
 0002:00000418       ??_7CModemStatus@@6B@      00112418     ModemStat.obj
 0002:0000041c       ??_C@_11LOCGONAA@?$AA?$AA@ 0011241c     ModemStat.obj
 0002:00000420       ??_C@_1FO@NDJHDAJC@?$AA?4?$AA?4?$AA?2?$AA?4?$AA?4?$AA?2?$AA?4?$AA?4?$AA?2?$AA?4?$AA?4?$AA?2?$AAR?$AAI?$AAL?$AAD?$AAr?$AAi?$AAv?$AAe?$AAr?$AA?2?$AAC?$AAo?$AAm?$AAm?$AAo?$AAn?$AA?2?$AAs?$AAr?$AAc@ 00112420     ModemStat.obj
 0002:00000480       ??_C@_1DG@LCAPKGOK@?$AAR?$AAI?$AAL?$AA_?$AAD?$AAe?$AAi?$AAn?$AAi?$AAt?$AAi?$AAa?$AAl?$AAi?$AAz?$AAe?$AA?5?$AAF?$AAa?$AAl?$AAi?$AAe?$AAd?$AA?5?$AA?$CF?$AAd?$AA?$AA@ 00112480     ModemStat.obj
 0002:000004b8       ??_C@_1GG@MLOAOBHO@?$AAU?$AAp?$AAd?$AAa?$AAt?$AAe?$AAC?$AAa?$AAl?$AAl?$AAT?$AAy?$AAp?$AAe?$AAA?$AAn?$AAd?$AAS?$AAt?$AAa?$AAt?$AAu?$AAs?$AA?5?$AAc?$AAa?$AAn?$AAn?$AAo?$AAt?$AA?5?$AAh@ 001124b8     ModemStat.obj
 0002:00000520       ??_C@_1JG@JMBAMLCB@?$AAI?$AAn?$AAv?$AAa?$AAl?$AAi?$AAd?$AA?5?$AAs?$AAt?$AAa?$AAt?$AAe?$AA?3?$AA?5?$AAm?$AA_?$AAC?$AAa?$AAl?$AAl?$AAT?$AAy?$AAp?$AAe?$AA?5?$AA?$DN?$AA?5?$AA?$CF?$AAd?$AA?5?$AAb@ 00112520     ModemStat.obj
 0002:000005b8       ??_C@_1FO@GFODOKOF@?$AAI?$AAn?$AAv?$AAa?$AAl?$AAi?$AAd?$AA?5?$AAs?$AAt?$AAa?$AAt?$AAe?$AA?3?$AA?5?$AAm?$AA_?$AAC?$AAa?$AAl?$AAl?$AAT?$AAy?$AAp?$AAe?$AA?5?$AA?$DN?$AA?5?$AA?$CF?$AAd?$AA?5?$AAb@ 001125b8     ModemStat.obj
 0002:00000618       ??_C@_1DK@CMAHCKEF@?$AAI?$AAn?$AAv?$AAa?$AAl?$AAi?$AAd?$AA?5?$AAc?$AAa?$AAl?$AAl?$AAE?$AAv?$AAe?$AAn?$AAt?$AAM?$AAa?$AAs?$AAk?$AA?5?$AA?$DN?$AA?5?$AA0?$AAx?$AA?$CF?$AAx?$AA?$AA@ 00112618     ModemStat.obj
 0002:00000654       ??_C@_1CI@CHFKALHP@?$AAU?$AAN?$AAC?$AAH?$AAG?$AA?0?$AA?5?$AAi?$AAn?$AAv?$AAa?$AAl?$AAi?$AAd?$AA?5?$AAc?$AAa?$AAs?$AAe?$AA?$AA@ 00112654     ModemStat.obj
 0002:00000680       ??_C@_1MA@HENCIANL@?$AAM?$AAi?$AAg?$AAh?$AAt?$AA?5?$AAw?$AAe?$AA?5?$AAf?$AAo?$AAr?$AAg?$AAe?$AAt?$AA?5?$AAt?$AAo?$AA?5?$AAs?$AAe?$AAt?$AA?5?$AAb?$AAS?$AAe?$AAn?$AAd?$AAE?$AAv?$AAe?$AAn@ 00112680     ModemStat.obj
 0002:00000740       ??_C@_1FC@IDICBMFI@?$AAU?$AAn?$AAh?$AAa?$AAn?$AAd?$AAl?$AAe?$AAd?$AA?5?$AAr?$AAe?$AAs?$AAu?$AAl?$AAt?$AA?5?$AAc?$AAa?$AAl?$AAl?$AAb?$AAa?$AAc?$AAk?$AA?5?$AAf?$AAo?$AAr?$AA?5?$AAI?$AAO@ 00112740     ModemStat.obj
 0002:00000798       ??_C@_1GG@DNHPCHDD@?$AAR?$AAe?$AAc?$AAe?$AAi?$AAv?$AAe?$AA?5?$AAR?$AAI?$AAL?$AA_?$AAR?$AAE?$AAS?$AAU?$AAL?$AAT?$AA_?$AAd?$AAw?$AAC?$AAo?$AAd?$AAe?$AA?5?$AA?$DN?$AA?5?$AA?$CF?$AAd?$AA?0?$AA?5@ 00112798     ModemStat.obj
 0002:00000800       ??_C@_1BAK@CBAAMEED@?$AAE?$AAr?$AAr?$AAo?$AAr?$AA?5?$AAi?$AAn?$AA?5?$AAR?$AAI?$AAL?$AA_?$AAA?$AAP?$AAI?$AA?3?$AAC?$AAm?$AAd?$AAI?$AAD?$AA?5?$AA?$DN?$AA?5?$AA?$CF?$AAd?$AA?0?$AAF?$AAu?$AAn?$AAc@ 00112800     ModemStat.obj
 0002:00000910       ??_C@_1BCM@KJPIKFNH@?$AAR?$AAI?$AAL?$AA?5?$AAR?$AAe?$AAs?$AAu?$AAl?$AAt?$AA?5?$AAr?$AAe?$AAc?$AAe?$AAi?$AAv?$AAe?$AAd?$AA?5?$AAi?$AAs?$AA?5?$AAf?$AAo?$AAr?$AA?5?$AAd?$AAi?$AAf?$AAf?$AAe@ 00112910     ModemStat.obj
 0002:00000a40       ??_C@_1KA@DAPMDLKE@?$AAS?$AAp?$AAe?$AAc?$AAu?$AAl?$AAa?$AAt?$AAe?$AA?5?$AAt?$AAh?$AAa?$AAt?$AA?5?$AAp?$AAr?$AAe?$AAv?$AAi?$AAo?$AAu?$AAs?$AA?5?$AAM?$AAo?$AAd?$AAe?$AAm?$AAS?$AAt?$AAa@ 00112a40     ModemStat.obj
 0002:00000ae0       ??_C@_1CI@DNMBCABB@?$AAE?$AAR?$AAR?$AA_?$AAR?$AAI?$AAL?$AA_?$AAA?$AAP?$AAI?$AA_?$AAT?$AAI?$AAM?$AAE?$AAO?$AAU?$AAT?$AA?$AA@ 00112ae0     ModemStat.obj
 0002:00000b08       ??_C@_1CI@IINHBIMO@?$AAE?$AAR?$AAR?$AA_?$AAR?$AAI?$AAL?$AA_?$AAA?$AAP?$AAI?$AA_?$AAF?$AAA?$AAI?$AAL?$AAU?$AAR?$AAE?$AA?$AA@ 00112b08     ModemStat.obj
 0002:00000b30       ??_C@_1LG@BCMGNPIC@?$AAE?$AAr?$AAr?$AAo?$AAr?$AA?5?$AAi?$AAn?$AA?5?$AAR?$AAI?$AAL?$AA_?$AAA?$AAP?$AAI?$AA?3?$AAC?$AAm?$AAd?$AAI?$AAD?$AA?5?$AA?$CI?$AAM?$AAo?$AAd?$AAe?$AAm?$AAS?$AAt?$AAa@ 00112b30     ModemStat.obj
 0002:00000be8       ??_C@_1BCC@LJKAGIOO@?$AAE?$AAr?$AAr?$AAo?$AAr?$AA?5?$AAi?$AAn?$AA?5?$AAR?$AAI?$AAL?$AA_?$AAA?$AAP?$AAI?$AA?3?$AAC?$AAm?$AAd?$AAI?$AAD?$AA?5?$AA?$CI?$AAM?$AAo?$AAd?$AAe?$AAm?$AAS?$AAt?$AAa@ 00112be8     ModemStat.obj
 0002:00000d10       ??_C@_1NG@HGDIBFPD@?$AAE?$AAr?$AAr?$AAo?$AAr?$AA?5?$AAi?$AAn?$AA?5?$AAR?$AAI?$AAL?$AA_?$AAA?$AAP?$AAI?$AA?3?$AAC?$AAm?$AAd?$AAI?$AAD?$AA?5?$AA?$CI?$AAM?$AAo?$AAd?$AAe?$AAm?$AAS?$AAt?$AAa@ 00112d10     ModemStat.obj
 0002:00000e20       ??_C@_1EM@MEJJDJJK@?$AAR?$AAI?$AAL?$AA?5?$AAr?$AAe?$AAs?$AAp?$AAo?$AAn?$AAs?$AAe?$AA?5?$AAc?$AAo?$AAn?$AAt?$AAa?$AAi?$AAn?$AAe?$AAr?$AA?5?$AAp?$AAa?$AAr?$AAa?$AAm?$AAs?$AA?5?$AAi?$AAn@ 00112e20     ModemStat.obj
 0002:00000e6c       ??_C@_1DM@GHAPEAGJ@?$AAR?$AAi?$AAl?$AA?5?$AAd?$AAr?$AAi?$AAv?$AAe?$AAr?$AA?5?$AAi?$AAs?$AA?5?$AAn?$AAo?$AAt?$AA?5?$AAi?$AAn?$AAi?$AAt?$AAi?$AAa?$AAl?$AAi?$AAz?$AAe?$AAd?$AA?$AA@ 00112e6c     ModemStat.obj
 0002:00000f78       ??_C@_1IA@IACALPMP@?$AAD?$AAS?$AA_?$AAG?$AAE?$AAT?$AA_?$AAP?$AAA?$AAC?$AAK?$AAE?$AAT?$AA_?$AAD?$AAA?$AAT?$AAA?$AA_?$AAS?$AAT?$AAA?$AAT?$AAU?$AAS?$AA_?$AAC?$AAI?$AAD?$AA?5?$AAf?$AAa@ 00112f78     ModemStat.obj
 0002:00000ff8       ??_C@_1JE@KLDDMDIG@?$AAG?$AAe?$AAt?$AAA?$AAd?$AAv?$AAa?$AAn?$AAc?$AAe?$AAd?$AAM?$AAe?$AAn?$AAu?$AAI?$AAn?$AAf?$AAo?$AA?5?$AAr?$AAe?$AAc?$AAe?$AAi?$AAv?$AAe?$AAs?$AA?5?$AAm?$AAi?$AAs@ 00112ff8     ModemStat.obj
 0002:00001090       ??_C@_1IO@BCBHHMPC@?$AAG?$AAe?$AAt?$AAP?$AAr?$AAo?$AAv?$AAi?$AAs?$AAi?$AAo?$AAn?$AAI?$AAn?$AAf?$AAo?$AA?5?$AAr?$AAe?$AAc?$AAe?$AAi?$AAv?$AAe?$AAs?$AA?5?$AAm?$AAi?$AAs?$AAm?$AAa?$AAt@ 00113090     ModemStat.obj
 0002:00001120       ??_C@_1DI@DIMDDOBO@?$AAU?$AAn?$AAa?$AAb?$AAl?$AAe?$AA?5?$AAt?$AAo?$AA?5?$AAg?$AAe?$AAt?$AA?5?$AAt?$AAh?$AAe?$AA?5?$AAP?$AAD?$AAS?$AAM?$AA?5?$AAD?$AAa?$AAt?$AAa?$AA?$AA@ 00113120     ModemStat.obj
 0002:00001158       ??_C@_1IM@BCLFBFJK@?$AAP?$AAa?$AAy?$AAl?$AAo?$AAa?$AAd?$AA?5?$AAf?$AAo?$AAr?$AA?5?$AAR?$AAI?$AAL?$AA_?$AAN?$AAO?$AAT?$AAI?$AAF?$AAY?$AA_?$AAI?$AAO?$AAT?$AAA?$AA_?$AAW?$AAA?$AAP?$AAP@ 00113158     ModemStat.obj
 0002:000011e4       ??_C@_1DK@PENNDGBL@?$AAI?$AAn?$AAv?$AAa?$AAl?$AAi?$AAd?$AA?5?$AA?5?$AAR?$AAI?$AAL?$AAI?$AAO?$AAT?$AAA?$AAS?$AAT?$AAA?$AAT?$AAU?$AAS?$AA?5?$AAD?$AAa?$AAt?$AAa?$AA?5?$AA?$AA@ 001131e4     ModemStat.obj
 0002:00001220       ??_C@_1EI@GEIIIKMC@?$AAP?$AAa?$AAy?$AAl?$AAo?$AAa?$AAd?$AA?5?$AAf?$AAo?$AAr?$AA?5?$AAR?$AAI?$AAL?$AA_?$AAN?$AAO?$AAT?$AAI?$AAF?$AAY?$AA_?$AAI?$AAO?$AAT?$AAA?$AA_?$AAS?$AAT?$AAA?$AAT@ 00113220     ModemStat.obj
 0002:00001268       ??_C@_1GI@DLFKOOLJ@?$AAR?$AAi?$AAl?$AAN?$AAo?$AAt?$AAi?$AAf?$AAy?$AAC?$AAa?$AAl?$AAl?$AAb?$AAa?$AAc?$AAk?$AA?$CI?$AA?$CJ?$AA?5?$AAR?$AAI?$AAL?$AA_?$AAN?$AAO?$AAT?$AAI?$AAF?$AAY?$AA_?$AAI@ 00113268     ModemStat.obj
 0002:000012d0       ??_C@_1DK@BPNHBMCK@?$AAI?$AAn?$AAv?$AAa?$AAl?$AAi?$AAd?$AA?5?$AA?5?$AAR?$AAI?$AAL?$AAT?$AAE?$AAC?$AAH?$AAH?$AAD?$AAR?$AAR?$AAR?$AAI?$AA?5?$AAD?$AAa?$AAt?$AAa?$AA?5?$AA?$AA@ 001132d0     ModemStat.obj
 0002:00001310       ??_C@_1JG@GOOFLPKI@?$AAP?$AAa?$AAy?$AAl?$AAo?$AAa?$AAd?$AA?5?$AAf?$AAo?$AAr?$AA?5?$AAR?$AAI?$AAL?$AA_?$AAN?$AAO?$AAT?$AAI?$AAF?$AAY?$AA_?$AAD?$AAE?$AAV?$AAS?$AAP?$AAC?$AA_?$AAT?$AAE@ 00113310     ModemStat.obj
 0002:000013a8       ??_C@_1EC@IFLCDBOE@?$AAI?$AAn?$AAv?$AAa?$AAl?$AAi?$AAd?$AA?5?$AA?5?$AAR?$AAI?$AAL?$AAT?$AAE?$AAC?$AAH?$AAH?$AAD?$AAR?$AAS?$AAE?$AAS?$AAS?$AAI?$AAO?$AAN?$AA?5?$AAD?$AAa?$AAt?$AAa?$AA?5@ 001133a8     ModemStat.obj
 0002:000013f0       ??_C@_1JO@FIJJCBGL@?$AAP?$AAa?$AAy?$AAl?$AAo?$AAa?$AAd?$AA?5?$AAf?$AAo?$AAr?$AA?5?$AAR?$AAI?$AAL?$AA_?$AAN?$AAO?$AAT?$AAI?$AAF?$AAY?$AA_?$AAD?$AAE?$AAV?$AAS?$AAP?$AAC?$AA_?$AAT?$AAE@ 001133f0     ModemStat.obj
 0002:00001490       ??_C@_1DO@FELKIJKN@?$AAI?$AAn?$AAv?$AAa?$AAl?$AAi?$AAd?$AA?5?$AA?5?$AAR?$AAI?$AAL?$AAT?$AAE?$AAC?$AAH?$AAH?$AAD?$AAR?$AAS?$AAT?$AAA?$AAT?$AAS?$AA?5?$AAD?$AAa?$AAt?$AAa?$AA?5?$AA?$AA@ 00113490     ModemStat.obj
 0002:000014d0       ??_C@_1JK@KJJNINIL@?$AAP?$AAa?$AAy?$AAl?$AAo?$AAa?$AAd?$AA?5?$AAf?$AAo?$AAr?$AA?5?$AAR?$AAI?$AAL?$AA_?$AAN?$AAO?$AAT?$AAI?$AAF?$AAY?$AA_?$AAD?$AAE?$AAV?$AAS?$AAP?$AAC?$AA_?$AAT?$AAE@ 001134d0     ModemStat.obj
 0002:00001570       ??_C@_1EA@LBEGGCKG@?$AAI?$AAn?$AAv?$AAa?$AAl?$AAi?$AAd?$AA?5?$AA?5?$AAR?$AAI?$AAL?$AAT?$AAE?$AAC?$AAH?$AAH?$AAD?$AAR?$AAS?$AAE?$AAC?$AAT?$AAO?$AAR?$AA?5?$AAD?$AAa?$AAt?$AAa?$AA?5?$AA?$AA@ 00113570     ModemStat.obj
 0002:000015b0       ??_C@_1JM@IFLHJBNA@?$AAP?$AAa?$AAy?$AAl?$AAo?$AAa?$AAd?$AA?5?$AAf?$AAo?$AAr?$AA?5?$AAR?$AAI?$AAL?$AA_?$AAN?$AAO?$AAT?$AAI?$AAF?$AAY?$AA_?$AAD?$AAE?$AAV?$AAS?$AAP?$AAC?$AA_?$AAT?$AAE@ 001135b0     ModemStat.obj
 0002:00001650       ??_C@_1EE@CPPOHGBH@?$AAI?$AAn?$AAv?$AAa?$AAl?$AAi?$AAd?$AA?5?$AA?5?$AAR?$AAI?$AAL?$AAT?$AAE?$AAC?$AAH?$AAH?$AAD?$AAR?$AAD?$AAR?$AAC?$AAC?$AAO?$AAV?$AAE?$AAR?$AA?5?$AAD?$AAa?$AAt?$AAa@ 00113650     ModemStat.obj
 0002:00001698       ??_C@_1KA@DDHPOBFP@?$AAP?$AAa?$AAy?$AAl?$AAo?$AAa?$AAd?$AA?5?$AAf?$AAo?$AAr?$AA?5?$AAR?$AAI?$AAL?$AA_?$AAN?$AAO?$AAT?$AAI?$AAF?$AAY?$AA_?$AAD?$AAE?$AAV?$AAS?$AAP?$AAC?$AA_?$AAT?$AAE@ 00113698     ModemStat.obj
 0002:00001738       ??_C@_1EA@JIOCKGIC@?$AAI?$AAn?$AAv?$AAa?$AAl?$AAi?$AAd?$AA?5?$AA?5?$AAR?$AAI?$AAL?$AAT?$AAE?$AAC?$AAH?$AAH?$AAD?$AAR?$AAD?$AAR?$AAC?$AAV?$AAA?$AAL?$AA?5?$AAD?$AAa?$AAt?$AAa?$AA?5?$AA?$AA@ 00113738     ModemStat.obj
 0002:00001778       ??_C@_1JM@JHEJBAIC@?$AAP?$AAa?$AAy?$AAl?$AAo?$AAa?$AAd?$AA?5?$AAf?$AAo?$AAr?$AA?5?$AAR?$AAI?$AAL?$AA_?$AAN?$AAO?$AAT?$AAI?$AAF?$AAY?$AA_?$AAD?$AAE?$AAV?$AAS?$AAP?$AAC?$AA_?$AAT?$AAE@ 00113778     ModemStat.obj
 0002:00001818       ??_C@_1EA@OJKLOCF@?$AAI?$AAn?$AAv?$AAa?$AAl?$AAi?$AAd?$AA?5?$AA?5?$AAR?$AAI?$AAL?$AAT?$AAE?$AAC?$AAH?$AAH?$AAD?$AAR?$AAA?$AAN?$AAA?$AAU?$AAT?$AAH?$AA?5?$AAD?$AAa?$AAt?$AAa?$AA?5?$AA?$AA@ 00113818     ModemStat.obj
 0002:00001858       ??_C@_1JM@JKDMKLCK@?$AAP?$AAa?$AAy?$AAl?$AAo?$AAa?$AAd?$AA?5?$AAf?$AAo?$AAr?$AA?5?$AAR?$AAI?$AAL?$AA_?$AAN?$AAO?$AAT?$AAI?$AAF?$AAY?$AA_?$AAD?$AAE?$AAV?$AAS?$AAP?$AAC?$AA_?$AAT?$AAE@ 00113858     ModemStat.obj
 0002:000018f8       ??_C@_1EC@IPEBJDAN@?$AAI?$AAn?$AAv?$AAa?$AAl?$AAi?$AAd?$AA?5?$AA?5?$AAR?$AAI?$AAL?$AAT?$AAE?$AAC?$AAH?$AAH?$AAD?$AAR?$AAC?$AAH?$AAA?$AAN?$AAN?$AAE?$AAL?$AA?5?$AAD?$AAa?$AAt?$AAa?$AA?5@ 001138f8     ModemStat.obj
 0002:00001940       ??_C@_1JO@EBMJCFKF@?$AAP?$AAa?$AAy?$AAl?$AAo?$AAa?$AAd?$AA?5?$AAf?$AAo?$AAr?$AA?5?$AAR?$AAI?$AAL?$AA_?$AAN?$AAO?$AAT?$AAI?$AAF?$AAY?$AA_?$AAD?$AAE?$AAV?$AAS?$AAP?$AAC?$AA_?$AAT?$AAE@ 00113940     ModemStat.obj
 0002:000019e0       ??_C@_1DO@OBAMNONH@?$AAI?$AAn?$AAv?$AAa?$AAl?$AAi?$AAd?$AA?5?$AA?5?$AAR?$AAI?$AAL?$AAT?$AAE?$AAC?$AAH?$AAH?$AAD?$AAR?$AAS?$AAT?$AAA?$AAT?$AAE?$AA?5?$AAD?$AAa?$AAt?$AAa?$AA?5?$AA?$AA@ 001139e0     ModemStat.obj
 0002:00001a20       ??_C@_1JK@BLFPHGLP@?$AAP?$AAa?$AAy?$AAl?$AAo?$AAa?$AAd?$AA?5?$AAf?$AAo?$AAr?$AA?5?$AAR?$AAI?$AAL?$AA_?$AAN?$AAO?$AAT?$AAI?$AAF?$AAY?$AA_?$AAD?$AAE?$AAV?$AAS?$AAP?$AAC?$AA_?$AAT?$AAE@ 00113a20     ModemStat.obj
 0002:00001abc       ??_C@_1DM@EBDNEKAJ@?$AAI?$AAn?$AAv?$AAa?$AAl?$AAi?$AAd?$AA?5?$AA?5?$AAR?$AAI?$AAL?$AAT?$AAE?$AAC?$AAH?$AAH?$AAD?$AAR?$AAP?$AAR?$AAE?$AAV?$AA?5?$AAD?$AAa?$AAt?$AAa?$AA?5?$AA?$AA@ 00113abc     ModemStat.obj
 0002:00001af8       ??_C@_1JI@IMCOAMGG@?$AAP?$AAa?$AAy?$AAl?$AAo?$AAa?$AAd?$AA?5?$AAf?$AAo?$AAr?$AA?5?$AAR?$AAI?$AAL?$AA_?$AAN?$AAO?$AAT?$AAI?$AAF?$AAY?$AA_?$AAD?$AAE?$AAV?$AAS?$AAP?$AAC?$AA_?$AAT?$AAE@ 00113af8     ModemStat.obj
 0002:00001b90       ??_C@_1EC@FGCOBHMO@?$AAI?$AAn?$AAv?$AAa?$AAl?$AAi?$AAd?$AA?5?$AA?5?$AAR?$AAI?$AAL?$AAM?$AAO?$AAD?$AAE?$AAM?$AAD?$AAE?$AAB?$AAU?$AAG?$AAI?$AAN?$AAF?$AAO?$AA?5?$AAD?$AAa?$AAt?$AAa?$AA?5@ 00113b90     ModemStat.obj
 0002:00001bd8       ??_C@_1JA@IEBHCCLO@?$AAP?$AAa?$AAy?$AAl?$AAo?$AAa?$AAd?$AA?5?$AAf?$AAo?$AAr?$AA?5?$AAR?$AAI?$AAL?$AA_?$AAN?$AAO?$AAT?$AAI?$AAF?$AAY?$AA_?$AAM?$AAO?$AAD?$AAE?$AAM?$AA_?$AAD?$AAB?$AAG@ 00113bd8     ModemStat.obj
 0002:00001c68       ??_C@_1DI@KINCGFNE@?$AAR?$AAI?$AAL?$AA_?$AAN?$AAO?$AAT?$AAI?$AAF?$AAY?$AA_?$AAM?$AAI?$AAN?$AA_?$AAA?$AAC?$AAT?$AAI?$AAV?$AAE?$AA_?$AAS?$AAT?$AAA?$AAT?$AAE?$AA?$AA@ 00113c68     ModemStat.obj
 0002:00001ca0       ??_C@_1CM@LCBGMALN@?$AAC?$AAa?$AAr?$AAr?$AAi?$AAe?$AAr?$AA?5?$AAI?$AAn?$AAd?$AAe?$AAx?$AA?5?$AAC?$AAh?$AAn?$AAa?$AAg?$AAe?$AAd?$AA?$AA@ 00113ca0     ModemStat.obj
 0002:00001ccc       ??_C@_1DC@IOHEHAAH@?$AAR?$AAI?$AAL?$AA_?$AAI?$AAn?$AAi?$AAt?$AAi?$AAa?$AAl?$AAi?$AAz?$AAe?$AA?5?$AAF?$AAa?$AAi?$AAl?$AAe?$AAd?$AA?5?$AA?$CF?$AAd?$AA?$AA@ 00113ccc     ModemStat.obj
 0002:00001d00       ??_C@_1FE@ELOMPPNC@?$AAM?$AAo?$AAd?$AAG?$AAe?$AAt?$AAC?$AAu?$AAr?$AAr?$AAe?$AAn?$AAt?$AAS?$AAy?$AAs?$AAt?$AAe?$AAm?$AAT?$AAy?$AAp?$AAe?$AA?5?$AAF?$AAa?$AAi?$AAl?$AAe?$AAd?$AA?5?$AAE@ 00113d00     ModemStat.obj
 0002:00001d58       ??_C@_1FC@NHJKOPIN@?$AAM?$AAo?$AAd?$AAG?$AAe?$AAt?$AAP?$AAa?$AAc?$AAk?$AAe?$AAt?$AAD?$AAa?$AAt?$AAa?$AAS?$AAt?$AAa?$AAt?$AAu?$AAs?$AA?5?$AAF?$AAa?$AAi?$AAl?$AAe?$AAd?$AA?5?$AAE?$AAr@ 00113d58     ModemStat.obj
 0002:00001db0       ??_C@_1EC@LGCAFOCL@?$AAM?$AAo?$AAd?$AAG?$AAe?$AAt?$AAC?$AAa?$AAl?$AAl?$AAL?$AAi?$AAs?$AAt?$AA?5?$AAF?$AAa?$AAi?$AAl?$AAe?$AAd?$AA?5?$AAE?$AAr?$AAr?$AAo?$AAr?$AA?5?$AA?$DN?$AA?5?$AA?$CF?$AAd@ 00113db0     ModemStat.obj
 0002:00001df8       ??_C@_1FG@LOOICFNM@?$AAM?$AAo?$AAd?$AAG?$AAe?$AAt?$AAR?$AAe?$AAg?$AAi?$AAs?$AAt?$AAr?$AAa?$AAt?$AAi?$AAo?$AAn?$AAS?$AAt?$AAa?$AAt?$AAu?$AAs?$AA?5?$AAF?$AAa?$AAi?$AAl?$AAe?$AAd?$AA?5@ 00113df8     ModemStat.obj
 0002:00001e50       ??_C@_1LI@DMNKNFJD@?$AAG?$AAe?$AAt?$AAE?$AAq?$AAu?$AAi?$AAp?$AAm?$AAe?$AAn?$AAt?$AAS?$AAt?$AAa?$AAt?$AAe?$AA?5?$AAE?$AAr?$AAr?$AAo?$AAr?$AA?5?$AA?$DN?$AA?5?$AA?$CF?$AAd?$AA?5?$AAo?$AAn?$AA?5@ 00113e50     ModemStat.obj
 0002:00001f40       ??_C@_1II@BKGIFOOG@?$AAG?$AAe?$AAt?$AAU?$AAs?$AAe?$AAr?$AAI?$AAd?$AAe?$AAn?$AAt?$AAi?$AAt?$AAy?$AA?5?$AAf?$AAa?$AAi?$AAl?$AAe?$AAd?$AA?3?$AA?5?$AAp?$AAd?$AAw?$AAR?$AAe?$AAs?$AAu?$AAl@ 00113f40     ModemStat.obj
 0002:00001fc8       ??_C@_1FO@HDMOIJ@?$AAU?$AAn?$AAk?$AAn?$AAo?$AAw?$AAn?$AA?5?$AAP?$AAo?$AAw?$AAe?$AAr?$AA?5?$AAS?$AAt?$AAa?$AAt?$AAe?$AA?5?$AAc?$AAa?$AAn?$AA?5?$AAn?$AAo?$AAt?$AA?5?$AAs?$AAe?$AAt?$AA?5@ 00113fc8     ModemStat.obj
 0002:00002028       ??_C@_1DG@CHMJAEKJ@?$AAc?$AAo?$AAu?$AAl?$AAd?$AA?5?$AAn?$AAo?$AAt?$AA?5?$AAp?$AAr?$AAe?$AAp?$AAa?$AAr?$AAe?$AA?5?$AAf?$AAo?$AAr?$AA?5?$AAd?$AAa?$AAt?$AAa?$AA?$AA@ 00114028     ModemStat.obj
 0002:00002060       ??_C@_1CC@CANGJEHL@?$AAS?$AAP?$AAC?$AA?5?$AAm?$AAo?$AAd?$AAe?$AA?5?$AAi?$AAs?$AA?5?$AA?$DN?$AA?5?$AA?$CF?$AAd?$AA?$AA@ 00114060     ModemStat.obj
 0002:00002088       ??_C@_1FO@GHONNAGG@?$AAU?$AAn?$AAa?$AAb?$AAl?$AAe?$AA?5?$AAt?$AAo?$AA?5?$AAg?$AAe?$AAt?$AA?5?$AAt?$AAh?$AAe?$AA?5?$AAv?$AAa?$AAl?$AAi?$AAd?$AA?5?$AAv?$AAe?$AAr?$AAs?$AAi?$AAo?$AAn?$AA?5@ 00114088     ModemStat.obj
 0002:000020e8       ??_C@_1IK@FNJOHAAD@?$AAG?$AAe?$AAt?$AAI?$AAO?$AAT?$AAA?$AAL?$AAo?$AAg?$AA?0?$AA?5?$AA?$CK?$AAp?$AAd?$AAw?$AAL?$AAe?$AAn?$AA?5?$AA?$DN?$AA?5?$AA?$CF?$AAd?$AA?5?$AAd?$AAi?$AAf?$AAf?$AAe?$AAr?$AAs@ 001140e8     ModemStat.obj
 0002:00002178       ??_C@_1FG@DKGILLMH@?$AAU?$AAn?$AAa?$AAb?$AAl?$AAe?$AA?5?$AAt?$AAo?$AA?5?$AAg?$AAe?$AAt?$AA?5?$AAt?$AAh?$AAe?$AA?5?$AAv?$AAa?$AAl?$AAi?$AAd?$AA?5?$AAP?$AAD?$AAP?$AA?5?$AAl?$AAi?$AAs?$AAt@ 00114178     ModemStat.obj
 0002:000021d0       ??_C@_1EC@PJAHBOIG@?$AAU?$AAn?$AAa?$AAb?$AAl?$AAe?$AA?5?$AAt?$AAo?$AA?5?$AAg?$AAe?$AAt?$AA?5?$AAt?$AAh?$AAe?$AA?5?$AAP?$AAD?$AAS?$AAM?$AA?5?$AAP?$AAA?$AA?5?$AAP?$AAa?$AAr?$AAa?$AAm?$AAs@ 001141d0     ModemStat.obj
 0002:00002218       ??_C@_1FI@FCPLCAMO@?$AAF?$AAa?$AAi?$AAl?$AA?5?$AAt?$AAo?$AA?5?$AAa?$AAl?$AAl?$AAo?$AAc?$AAa?$AAt?$AAe?$AA?5?$AAm?$AAe?$AAm?$AAo?$AAr?$AAy?$AA?5?$AAf?$AAo?$AAr?$AA?5?$AA?$CK?$AAt?$AAC?$AAh@ 00114218     ModemStat.obj
 0002:00002270       ??_C@_1BI@GCDMFKAA@?$AAN?$AAO?$AA?5?$AAC?$AAA?$AAR?$AAR?$AAI?$AAE?$AAR?$AA?$AN?$AA?$AA@ 00114270     ModemStat.obj
 0002:00002288       ??_C@_1BE@LAJFGDPL@?$AA?$DN?$AA?5?$AAS?$AAT?$AAA?$AAT?$AAU?$AAS?$AA?$DN?$AA?$AA@ 00114288     ModemStat.obj
 0002:0000229c       ??_C@_0O@HBJJMLDE@AT?$CBGSTATUS?$DP?$AN?6?$AA@ 0011429c     ModemStat.obj
 0002:000022ac       ??_C@_1O@JDLOHAN@?$AAD?$AAe?$AAl?$AAe?$AAt?$AAe?$AA?$AA@ 001142ac     stdafx.obj
 0002:000022bc       ??_C@_1BC@GCKHIPE@?$AAN?$AAo?$AAR?$AAe?$AAm?$AAo?$AAv?$AAe?$AA?$AA@ 001142bc     stdafx.obj
 0002:000022d0       ??_C@_1BI@JFAIJMHL@?$AAF?$AAo?$AAr?$AAc?$AAe?$AAR?$AAe?$AAm?$AAo?$AAv?$AAe?$AA?$AA@ 001142d0     stdafx.obj
 0002:000022e8       ??_C@_17LLMMEOJD@?$AAV?$AAa?$AAl?$AA?$AA@ 001142e8     stdafx.obj
 0002:000022f0       ??_C@_13OPKGLAFF@?$AAB?$AA?$AA@ 001142f0     stdafx.obj
 0002:000022f4       ??_C@_13MKMNOPIJ@?$AAD?$AA?$AA@ 001142f4     stdafx.obj
 0002:000022f8       ??_C@_13LHMFKAAD@?$AAM?$AA?$AA@ 001142f8     stdafx.obj
 0002:000022fc       ??_C@_13HADIAKP@?$AAS?$AA?$AA@ 001142fc     stdafx.obj
 0002:00002db0       ??_C@_1EI@PPIEGFMO@?$AAT?$AAh?$AAe?$AA?5?$AAl?$AAa?$AAs?$AAt?$AA?5?$AAL?$AAo?$AAg?$AA?5?$AAt?$AAo?$AA?5?$AAk?$AAi?$AAl?$AAl?$AA?5?$AAt?$AAh?$AAe?$AA?5?$AAl?$AAo?$AAg?$AA?5?$AAt?$AAh?$AAr@ 00114db0     SW_Log.obj
 0002:00002df8       ??_C@_1BG@JDINCLPI@?$AAS?$AAS?$AA_?$AAL?$AAo?$AAg?$AA?4?$AAl?$AAo?$AAg?$AA?$AA@ 00114df8     SW_Log.obj
 0002:00002e10       ??_C@_1CC@HCGICOJF@?$AAD?$AAe?$AAf?$AAa?$AAu?$AAl?$AAt?$AA?5?$AAL?$AAo?$AAg?$AA?5?$AAF?$AAi?$AAl?$AAe?$AA?$AA@ 00114e10     SW_Log.obj
 0002:00002e34       ??_C@_1O@FHLFJINA@?$AAS?$AAS?$AA_?$AAL?$AAo?$AAg?$AA?$AA@ 00114e34     SW_Log.obj
 0002:00002e44       ??_C@_1CO@FFGDIOPC@?$AAS?$AAi?$AAz?$AAe?$AA?5?$AA?9?$AA?5?$AA?5?$AA?5?$AAL?$AAo?$AAg?$AA?5?$AAF?$AAi?$AAl?$AAe?$AA?5?$AAS?$AAi?$AAz?$AAe?$AA?$AA@ 00114e44     SW_Log.obj
 0002:00002e74       ??_C@_1DE@NODGMBEK@?$AAF?$AAi?$AAl?$AAt?$AAe?$AAr?$AA?5?$AA?9?$AA?5?$AAS?$AAt?$AAa?$AAt?$AAu?$AAs?$AA?5?$AAC?$AAo?$AAm?$AAp?$AAL?$AAe?$AAv?$AAe?$AAl?$AA?$AA@ 00114e74     SW_Log.obj
 0002:00002ea8       ??_C@_1CI@BCFHDEIK@?$AAR?$AAe?$AAt?$AAa?$AAi?$AAl?$AA?5?$AAD?$AAe?$AAb?$AAu?$AAg?$AA?5?$AAE?$AAn?$AAa?$AAb?$AAl?$AAe?$AA?$AA@ 00114ea8     SW_Log.obj
 0002:00002ed0       ??_C@_1DC@BCJHBIKP@?$AAF?$AAi?$AAl?$AAt?$AAe?$AAr?$AA?5?$AA?9?$AA?5?$AAS?$AAt?$AAa?$AAt?$AAu?$AAs?$AA?5?$AAL?$AAo?$AAg?$AAL?$AAe?$AAv?$AAe?$AAl?$AA?$AA@ 00114ed0     SW_Log.obj
 0002:00002f04       ??_C@_1BI@MLPMOOF@?$AAD?$AAi?$AAs?$AAp?$AAl?$AAa?$AAy?$AA?5?$AAM?$AAe?$AAm?$AA?$AA@ 00114f04     SW_Log.obj
 0002:00002f20       ??_C@_1FK@KFPOPMD@?$AAG?$AAe?$AAt?$AAR?$AAe?$AAg?$AAV?$AAa?$AAl?$AAu?$AAe?$AA?5?$AAr?$AAe?$AAt?$AAu?$AAr?$AAn?$AAe?$AAd?$AA?5?$AA?$CF?$AAl?$AAu?$AA?5?$AAd?$AAw?$AAD?$AAi?$AAs?$AAp?$AAl@ 00114f20     SW_Log.obj
 0002:00002f7c       ??_C@_17LLLMIFAB@?$AAL?$AAo?$AAg?$AA?$AA@ 00114f7c     SW_Log.obj
 0002:00002f84       ??_C@_17KKLPNNMB@?$AAC?$AAO?$AAM?$AA?$AA@ 00114f84     SW_Log.obj
 0002:00002f90       ??_C@_1FA@FCCHEPJI@?$AA?6?$AA?$AN?$AAF?$AAa?$AAi?$AAl?$AA?5?$AAt?$AAo?$AA?5?$AAC?$AAr?$AAe?$AAa?$AAt?$AAe?$AAF?$AAi?$AAl?$AAe?$AA?5?$AAf?$AAo?$AAr?$AA?5?$AAt?$AAh?$AAe?$AA?5?$AAl?$AAo?$AAg@ 00114f90     SW_Log.obj
 0002:00002fe0       ??_C@_1CK@NCJHIFHF@?$AAE?$AAr?$AAr?$AA?5?$AA?$DN?$AA?5?$AA0?$AAx?$AA?$CF?$AAx?$AA?0?$AA?5?$AAh?$AA?5?$AA?$DN?$AA?5?$AA0?$AAx?$AA?$CF?$AAx?$AA?$AA@ 00114fe0     SW_Log.obj
 0002:00003010       ??_C@_1HC@BHPNGIIO@?$AAC?$AAr?$AAe?$AAa?$AAt?$AAe?$AAF?$AAi?$AAl?$AAe?$AA?5?$AAf?$AAo?$AAr?$AA?5?$AAt?$AAh?$AAe?$AA?5?$AAe?$AAx?$AAi?$AAs?$AAt?$AAi?$AAn?$AAg?$AA?5?$AAl?$AAo?$AAg?$AA?5@ 00115010     SW_Log.obj
 0002:00003084       ??_C@_1DO@PFEABMDF@?$AA?$CB?$AA?$CB?$AA?$CB?$AAL?$AAo?$AAg?$AA?5?$AAf?$AAu?$AAl?$AAl?$AA?3?$AA?5?$AAc?$AAo?$AAu?$AAn?$AAt?$AA?5?$AA?$DN?$AA?5?$AA?$CF?$AAd?$AA?5?$AA?$EA?$AA?5?$AA?$CF?$AAs?$AA?$AN?$AA?6?$AA?$AA@ 00115084     SW_Log.obj
 0002:000030c4       ??_C@_1BA@LHCPJILL@?$AAO?$AAl?$AAd?$AA?4?$AAl?$AAo?$AAg?$AA?$AA@ 001150c4     SW_Log.obj
 0002:000030d4       ??_C@_19JFPGGDCL@?$AA?4?$AAl?$AAo?$AAg?$AA?$AA@ 001150d4     SW_Log.obj
 0002:000030e0       ??_C@_1DC@IPGAJIPB@?$AAW?$AAr?$AAi?$AAt?$AAe?$AAM?$AAs?$AAg?$AAQ?$AAu?$AAe?$AAu?$AAe?$AA?5?$AAE?$AAr?$AAr?$AA?5?$AA?$DN?$AA?5?$AA0?$AAx?$AA?$CF?$AAx?$AA?$AA@ 001150e0     SW_Log.obj
 0002:00003114       ??_C@_13HOIJIPNN@?$AA?5?$AA?$AA@ 00115114     SW_Log.obj
 0002:00003118       ??_C@_1M@MGIHBMCI@?$AAT?$AAR?$AAA?$AAC?$AAE?$AA?$AA@ 00115118     SW_Log.obj
 0002:00003124       ??_C@_1BA@KPCCLDOC@?$AAW?$AAA?$AAR?$AAN?$AAI?$AAN?$AAG?$AA?$AA@ 00115124     SW_Log.obj
 0002:00003134       ??_C@_13CGOKJPIL@?$AA?1?$AA?$AA@ 00115134     SW_Log.obj
 0002:00003138       ??_C@_1BC@IHPPMOFN@?$AAC?$AAR?$AAI?$AAT?$AAI?$AAC?$AAA?$AAL?$AA?$AA@ 00115138     SW_Log.obj
 0002:0000314c       ??_C@_1BA@HMOCDLBP@?$AAV?$AAE?$AAR?$AAS?$AAI?$AAO?$AAN?$AA?$AA@ 0011514c     SW_Log.obj
 0002:0000315c       ??_C@_1BM@MHBJMCAA@?$AAU?$AAP?$AA?5?$AA?$CF?$AA0?$AAX?$AA?5?$AAA?$AAB?$AA?5?$AA?$CF?$AA0?$AAX?$AA?$AA@ 0011515c     SW_Log.obj
 0002:00003178       ??_C@_1DO@ELJPEGAK@?$AA?$CF?$AA0?$AA2?$AAd?$AA?3?$AA?$CF?$AA0?$AA2?$AAd?$AA?3?$AA?$CF?$AA0?$AA2?$AAd?$AA?0?$AA?5?$AA?$CF?$AA0?$AA2?$AAd?$AA?4?$AA?$CF?$AA0?$AA2?$AAd?$AA?4?$AA?$CF?$AA0?$AA2?$AAd?$AA?$AA@ 00115178     SW_Log.obj
 0002:000031b8       ??_C@_1CK@LBLFIIHF@?$AA?$CF?$AAs?$AA?7?$AA?$CF?$AAs?$AA?7?$AA?$CF?$AAs?$AA?7?$AA?$CF?$AAd?$AA?7?$AA?$CF?$AA8?$AAs?$AA?7?$AA?$CF?$AAs?$AA?$AN?$AA?6?$AA?$AA@ 001151b8     SW_Log.obj
 0002:000031e4       ??_C@_1CM@HCDOAHOI@?$AAS?$AAW?$AA?5?$AAL?$AAo?$AAg?$AA?5?$AAM?$AAs?$AAg?$AA?5?$AAQ?$AAu?$AAe?$AAu?$AAe?$AA?5?$AAN?$AAa?$AAm?$AAe?$AA?$AA@ 001151e4     SW_Log.obj
 0002:00003210       ??_C@_1CO@MCIJBMIA@?$AAS?$AAW?$AA?5?$AAS?$AAS?$AAL?$AAo?$AAg?$AA?5?$AAW?$AAr?$AAi?$AAt?$AAi?$AAn?$AAg?$AA?5?$AAM?$AAu?$AAt?$AAe?$AAx?$AA?$AA@ 00115210     SW_Log.obj
 0002:00003280       ??_C@_13OHNMPHJM@?$AA?$FN?$AA?$AA@ 00115280     SW_Log_Include.obj
 0002:00003288       ??_C@_1IA@GJIGFKKM@?$AA?5?$AA?5?$AA?5?$AA?5?$AA?5?$AA?5?$AA?5?$AA?5?$AA?5?$AA?5?$AA?5?$AA?5?$AA?5?$AA?5?$AA?5?$AA?5?$AA?5?$AA?5?$AA?5?$AA?5?$AA?5?$AA?5?$AA?5?$AA?5?$AA?5?$AA?5?$AA?5?$AA?5?$AA?5?$AA?5?$AA?5?$AA?5@ 00115288     SW_Log_Include.obj
 0002:00003308       ??_C@_1M@OMOAGDNC@?$AA?$CF?$AA0?$AA2?$AAx?$AA?5?$AA?$AA@ 00115308     SW_Log_Include.obj
 0002:00003314       ??_C@_1BE@DFBIOGAO@?$AA?$DO?$AA?$DO?$AA?$CF?$AAd?$AA?$DO?$AA?$DO?$AA?5?$AA?$FL?$AA?5?$AA?$AA@ 00115314     SW_Log_Include.obj
 0002:00003328       ??_C@_17GMPJMPF@?$AA?$CF?$AAs?$AA?5?$AA?$AA@ 00115328     SW_Log_Include.obj
 0002:00003330       ??_C@_1CK@EGKKKNHB@?$AA?4?$AA?2?$AAS?$AAW?$AA_?$AAL?$AAo?$AAg?$AA_?$AAI?$AAn?$AAc?$AAl?$AAu?$AAd?$AAe?$AA?4?$AAc?$AAp?$AAp?$AA?$AA@ 00115330     SW_Log_Include.obj
 0002:0000335c       ??_C@_1CO@JIFOJHDN@?$AA?$CF?$AAs?$AA?5?$AA?4?$AA?4?$AA?4?$AA?5?$AAb?$AAu?$AAt?$AA?5?$AAl?$AAe?$AAn?$AAg?$AAt?$AAh?$AA?5?$AAi?$AAs?$AA?5?$AA0?$AA?$AA@ 0011535c     SW_Log_Include.obj
 0002:00003390       ??_C@_1GI@OJCPLOI@?$AA?$DO?$AA?$DO?$AA?$CF?$AAd?$AA?$DO?$AA?$DO?$AA?5?$AAN?$AAo?$AAw?$AA?5?$AAd?$AAu?$AAm?$AAp?$AAi?$AAn?$AAg?$AA?5?$AAt?$AAh?$AAe?$AA?5?$AAb?$AAu?$AAf?$AAf?$AAe?$AAr?$AA?5?$AAo?$AAf@ 00115390     SW_Log_Include.obj
 0002:000033f8       ??_C@_1CM@MEPMHBMB@?$AA?$DO?$AA?$DO?$AA?$CF?$AAd?$AA?$DO?$AA?$DO?$AA?5?$AA?$CF?$AAs?$AA?5?$AA?3?$AA?5?$AA?$CF?$AAd?$AA?5?$AAD?$AAa?$AAt?$AAa?$AA?3?$AA?5?$AA?$AA@ 001153f8     SW_Log_Include.obj
 0002:00003428       ??_C@_1GK@DBPEKJDK@?$AAS?$AAS?$AAL?$AAo?$AAg?$AA?5?$AAp?$AAr?$AAo?$AAb?$AAl?$AAe?$AAm?$AA?3?$AA?5?$AAR?$AAe?$AAg?$AAQ?$AAu?$AAe?$AAr?$AAy?$AAV?$AAa?$AAl?$AAu?$AAe?$AAE?$AAx?$AA?5?$AA?$CF@ 00115428     SW_Registrykey.obj
 0002:00003498       ??_C@_1IK@JELLMGK@?$AAS?$AAS?$AAL?$AAo?$AAg?$AA?5?$AAp?$AAr?$AAo?$AAb?$AAl?$AAe?$AAm?$AA?3?$AA?5?$AAR?$AAe?$AAg?$AAQ?$AAu?$AAe?$AAr?$AAy?$AAV?$AAa?$AAl?$AAu?$AAe?$AAE?$AAx?$AA?5?$AA?$CF@ 00115498     SW_Registrykey.obj
 0002:000035d8       ??_C@_1HO@CADMMIFD@?$AAS?$AAS?$AAL?$AAo?$AAg?$AA?5?$AAp?$AAr?$AAo?$AAb?$AAl?$AAe?$AAm?$AA?3?$AA?5?$AAS?$AAS?$AAL?$AAo?$AAg?$AA?5?$AAp?$AAr?$AAo?$AAb?$AAl?$AAe?$AAm?$AA?3?$AA?5?$AAQ?$AAu@ 001155d8     SW_Registrykey.obj
 0002:00003658       ??_C@_1IM@NNDKMKB@?$AAS?$AAS?$AAL?$AAo?$AAg?$AA?5?$AAp?$AAr?$AAo?$AAb?$AAl?$AAe?$AAm?$AA?3?$AA?5?$AAS?$AAS?$AAL?$AAo?$AAg?$AA?5?$AAp?$AAr?$AAo?$AAb?$AAl?$AAe?$AAm?$AA?3?$AA?5?$AAO?$AAp@ 00115658     SW_Registrykey.obj
 0002:00003850       ??_C@_1KA@ONCODNJL@?$AAS?$AAS?$AAL?$AAo?$AAg?$AA?5?$AAS?$AAW?$AAA?$AAI?$AA_?$AAG?$AAe?$AAt?$AAR?$AAe?$AAg?$AAV?$AAa?$AAl?$AAu?$AAe?$AA?5?$AAp?$AAr?$AAo?$AAb?$AAl?$AAe?$AAm?$AA?3?$AA?5@ 00115850     SW_Registrykey.obj
 0002:000038f0       ??_C@_1JK@NKOBMIHF@?$AAS?$AAS?$AAL?$AAo?$AAg?$AA?5?$AAS?$AAW?$AAA?$AAI?$AA_?$AAG?$AAe?$AAt?$AAR?$AAe?$AAg?$AAV?$AAa?$AAl?$AAu?$AAe?$AA?5?$AAp?$AAr?$AAo?$AAb?$AAl?$AAe?$AAm?$AA?3?$AA?5@ 001158f0     SW_Registrykey.obj
 0002:0000398c       ??_C@_1DK@DFOPCCDF@?$AAS?$AAo?$AAf?$AAt?$AAw?$AAa?$AAr?$AAe?$AA?2?$AAS?$AAi?$AAe?$AAr?$AAr?$AAa?$AA?5?$AAW?$AAi?$AAr?$AAe?$AAl?$AAe?$AAs?$AAs?$AA?5?$AAI?$AAn?$AAc?$AA?$AA@ 0011598c     SW_Registrykey.obj
 0002:000039c8       ??_C@_17CHCGIDNB@?$AA?$CF?$AAs?$AA?2?$AA?$AA@ 001159c8     SW_Registrykey.obj
 0002:00003d58       ??_C@_1BBI@KEIMOGPE@?$AA?$DM?$AAw?$AAa?$AAp?$AA?9?$AAp?$AAr?$AAo?$AAv?$AAi?$AAs?$AAi?$AAo?$AAn?$AAi?$AAn?$AAg?$AAd?$AAo?$AAc?$AA?$DO?$AA?$DM?$AAc?$AAh?$AAa?$AAr?$AAa?$AAc?$AAt?$AAe?$AAr?$AAi@ 00115d58     Utilities.obj
 0002:00003e70       ??_C@_1BBE@OEFMELPN@?$AA?$DM?$AAw?$AAa?$AAp?$AA?9?$AAp?$AAr?$AAo?$AAv?$AAi?$AAs?$AAi?$AAo?$AAn?$AAi?$AAn?$AAg?$AAd?$AAo?$AAc?$AA?$DO?$AA?$DM?$AAc?$AAh?$AAa?$AAr?$AAa?$AAc?$AAt?$AAe?$AAr?$AAi@ 00115e70     Utilities.obj
 0002:00003f88       ??_C@_1BBA@BNGDPGCH@?$AA?$DM?$AAw?$AAa?$AAp?$AA?9?$AAp?$AAr?$AAo?$AAv?$AAi?$AAs?$AAi?$AAo?$AAn?$AAi?$AAn?$AAg?$AAd?$AAo?$AAc?$AA?$DO?$AA?$DM?$AAc?$AAh?$AAa?$AAr?$AAa?$AAc?$AAt?$AAe?$AAr?$AAi@ 00115f88     Utilities.obj
 0002:00004098       ??_C@_1BAM@MDABPJEJ@?$AA?$DM?$AAw?$AAa?$AAp?$AA?9?$AAp?$AAr?$AAo?$AAv?$AAi?$AAs?$AAi?$AAo?$AAn?$AAi?$AAn?$AAg?$AAd?$AAo?$AAc?$AA?$DO?$AA?$DM?$AAc?$AAh?$AAa?$AAr?$AAa?$AAc?$AAt?$AAe?$AAr?$AAi@ 00116098     Utilities.obj
 0002:000041a8       ??_C@_1BBK@BJFAAOKO@?$AA?$DM?$AAw?$AAa?$AAp?$AA?9?$AAp?$AAr?$AAo?$AAv?$AAi?$AAs?$AAi?$AAo?$AAn?$AAi?$AAn?$AAg?$AAd?$AAo?$AAc?$AA?$DO?$AA?$DM?$AAc?$AAh?$AAa?$AAr?$AAa?$AAc?$AAt?$AAe?$AAr?$AAi@ 001161a8     Utilities.obj
 0002:000042c8       ??_C@_1BBE@BFBNLOMN@?$AA?$DM?$AAw?$AAa?$AAp?$AA?9?$AAp?$AAr?$AAo?$AAv?$AAi?$AAs?$AAi?$AAo?$AAn?$AAi?$AAn?$AAg?$AAd?$AAo?$AAc?$AA?$DO?$AA?$DM?$AAc?$AAh?$AAa?$AAr?$AAa?$AAc?$AAt?$AAe?$AAr?$AAi@ 001162c8     Utilities.obj
 0002:000043e0       ??_C@_1EHG@NEIJDEAF@?$AA?$DM?$AAw?$AAa?$AAp?$AA?9?$AAp?$AAr?$AAo?$AAv?$AAi?$AAs?$AAi?$AAo?$AAn?$AAi?$AAn?$AAg?$AAd?$AAo?$AAc?$AA?$DO?$AA?$DM?$AAc?$AAh?$AAa?$AAr?$AAa?$AAc?$AAt?$AAe?$AAr?$AAi@ 001163e0     Utilities.obj
 0002:00004858       ??_C@_1EGG@GIJGENHJ@?$AA?$DM?$AAw?$AAa?$AAp?$AA?9?$AAp?$AAr?$AAo?$AAv?$AAi?$AAs?$AAi?$AAo?$AAn?$AAi?$AAn?$AAg?$AAd?$AAo?$AAc?$AA?$DO?$AA?$DM?$AAc?$AAh?$AAa?$AAr?$AAa?$AAc?$AAt?$AAe?$AAr?$AAi@ 00116858     Utilities.obj
 0002:00004cc0       ??_C@_1HOO@GPHFMKKP@?$AA?$DM?$AAw?$AAa?$AAp?$AA?9?$AAp?$AAr?$AAo?$AAv?$AAi?$AAs?$AAi?$AAo?$AAn?$AAi?$AAn?$AAg?$AAd?$AAo?$AAc?$AA?$DO?$AA?$DM?$AAc?$AAh?$AAa?$AAr?$AAa?$AAc?$AAt?$AAe?$AAr?$AAi@ 00116cc0     Utilities.obj
 0002:000054b0       ??_C@_1CLO@EKODNOLM@?$AA?$DM?$AAw?$AAa?$AAp?$AA?9?$AAp?$AAr?$AAo?$AAv?$AAi?$AAs?$AAi?$AAo?$AAn?$AAi?$AAn?$AAg?$AAd?$AAo?$AAc?$AA?$DO?$AA?$DM?$AAc?$AAh?$AAa?$AAr?$AAa?$AAc?$AAt?$AAe?$AAr?$AAi@ 001174b0     Utilities.obj
 0002:000057bc       ??_C@_1BE@LAEKLHFJ@?$AAD?$AAa?$AAt?$AAe?$AA?$CG?$AAT?$AAi?$AAm?$AAe?$AA?$AA@ 001177bc     Utilities.obj
 0002:000057d0       ??_C@_1EK@BDCCKJKH@?$AAP?$AAr?$AAo?$AAd?$AAu?$AAc?$AAt?$AA?5?$AAN?$AAa?$AAm?$AAe?$AA?3?$AA?5?$AA?$CF?$AAs?$AA?5?$AAP?$AAr?$AAo?$AAd?$AAu?$AAc?$AAt?$AA?5?$AAV?$AAe?$AAr?$AAs?$AAi?$AAo?$AAn@ 001177d0     Utilities.obj
 0002:00005820       ??_C@_1FA@MMIAEGIF@?$AA?5?$AAD?$AAa?$AAt?$AAe?$AAT?$AAi?$AAm?$AAe?$AA?3?$AA?5?$AA?$CF?$AAs?$AA?5?$AAM?$AAo?$AAd?$AAu?$AAl?$AAe?$AA?5?$AAN?$AAa?$AAm?$AAe?$AA?5?$AAa?$AAn?$AAd?$AA?5?$AAP?$AAa@ 00117820     Utilities.obj
 0002:00005870       ??_C@_1M@KEKDJCFI@?$AA?$CF?$AAs?$AA?$CF?$AAd?$AA?3?$AA?$AA@ 00117870     Utilities.obj
 0002:0000587c       ??_C@_1BC@MIOHADKO@?$AAB?$AAa?$AAu?$AAd?$AAR?$AAa?$AAt?$AAe?$AA?$AA@ 0011787c     Utilities.obj
 0002:00005890       ??_C@_1O@GBAEOCCH@?$AAP?$AAr?$AAe?$AAf?$AAi?$AAx?$AA?$AA@ 00117890     Utilities.obj
 0002:000058a0       ??_C@_1M@EENNDIOJ@?$AAI?$AAn?$AAd?$AAe?$AAx?$AA?$AA@ 001178a0     Utilities.obj
 0002:000058ac       ??_C@_1BK@BIHJIGMO@?$AAR?$AAI?$AAL?$AA?2?$AAC?$AAD?$AAM?$AAA?$AAD?$AAa?$AAt?$AAa?$AA?$AA@ 001178ac     Utilities.obj
 0002:000058c8       ??_C@_19PNHLOHBK@?$AAR?$AAU?$AAI?$AAM?$AA?$AA@ 001178c8     Utilities.obj
 0002:000058d4       ??_C@_17FKOBBBNL@?$AAG?$AAS?$AAM?$AA?$AA@ 001178d4     Utilities.obj
 0002:000058dc       ??_C@_15JCPNBDBO@?$AAS?$AAW?$AA?$AA@ 001178dc     Utilities.obj
 0002:000058e4       ??_C@_17PCFLMGFN@?$AAV?$AAZ?$AAW?$AA?$AA@ 001178e4     Utilities.obj
 0002:000058ec       ??_C@_1DK@MMCNDJKH@?$AAC?$AAa?$AAr?$AAr?$AAi?$AAe?$AAr?$AA?5?$AAN?$AAa?$AAm?$AAe?$AA?5?$AAi?$AAs?$AA?5?$AA?$CF?$AAs?$AA?5?$AAl?$AAe?$AAn?$AA?5?$AAi?$AAs?$AA?5?$AA?$CF?$AAd?$AA?$AA@ 001178ec     Utilities.obj
 0002:00005928       ??_C@_17JPIPALNO@?$AAP?$AAC?$AAS?$AA?$AA@ 00117928     Utilities.obj
 0002:00005930       ??_C@_1GG@CEHGPBGP@?$AAU?$AAn?$AAa?$AAb?$AAl?$AAe?$AA?5?$AAt?$AAo?$AA?5?$AAo?$AAp?$AAe?$AAn?$AA?5?$AAt?$AAh?$AAe?$AA?5?$AAr?$AAe?$AAg?$AAi?$AAs?$AAt?$AAr?$AAy?$AA?5?$AAk?$AAe?$AAy?$AA?5@ 00117930     Utilities.obj
 0002:00005998       ??_C@_1BM@CHNBANCA@?$AAC?$AAa?$AAr?$AAr?$AAi?$AAe?$AAr?$AAS?$AAu?$AAf?$AAf?$AAi?$AAx?$AA?$AA@ 00117998     Utilities.obj
 0002:000059b4       ??_C@_1BI@FJLDDKCH@?$AAN?$AAe?$AAt?$AAw?$AAo?$AAr?$AAk?$AAT?$AAy?$AAp?$AAe?$AA?$AA@ 001179b4     Utilities.obj
 0002:000059cc       ??_C@_1CO@PFFMHNAH@?$AAS?$AAo?$AAf?$AAt?$AAw?$AAa?$AAr?$AAe?$AA?2?$AAM?$AAi?$AAc?$AAr?$AAo?$AAs?$AAo?$AAf?$AAt?$AA?2?$AAR?$AAI?$AAL?$AA?$AA@ 001179cc     Utilities.obj
 0002:000059fc       ??_C@_1BO@HEDCJKAP@?$AAA?$AAu?$AAt?$AAo?$AAU?$AAp?$AAd?$AAa?$AAt?$AAe?$AAT?$AAi?$AAm?$AAe?$AA?$AA@ 001179fc     Utilities.obj
 0002:00005a1c       ??_C@_1O@GINMMDNN@?$AAS?$AAy?$AAs?$AAt?$AAe?$AAm?$AA?$AA@ 00117a1c     Utilities.obj
 0002:00005a2c       ??_C@_1CC@KIKAECNH@?$AAA?$AAu?$AAt?$AAo?$AAU?$AAp?$AAd?$AAa?$AAt?$AAe?$AAT?$AAi?$AAm?$AAe?$AAU?$AAI?$AA?$AA@ 00117a2c     Utilities.obj
 0002:00005a50       ??_C@_1BE@OIBEOKIJ@?$AAR?$AAo?$AAa?$AAm?$AAG?$AAu?$AAa?$AAr?$AAd?$AA?$AA@ 00117a50     Utilities.obj
 0002:00005a64       ??_C@_1CE@NOHEPHEB@?$AAD?$AAi?$AAs?$AAa?$AAb?$AAl?$AAe?$AAA?$AAu?$AAt?$AAo?$AAA?$AAc?$AAt?$AAW?$AAi?$AAz?$AA?$AA@ 00117a64     Utilities.obj
 0002:00005a88       ??_C@_1O@JGODHDHF@?$AAM?$AAD?$AAN?$AAL?$AAe?$AAn?$AA?$AA@ 00117a88     Utilities.obj
 0002:00005a98       ??_C@_1BO@JIDEGKKH@?$AAC?$AAa?$AAr?$AAr?$AAi?$AAe?$AAr?$AAP?$AAr?$AAo?$AAd?$AAu?$AAc?$AAt?$AA?$AA@ 00117a98     Utilities.obj
 0002:00005ab8       ??_C@_1BK@HNGGBJHI@?$AAD?$AAi?$AAs?$AAa?$AAb?$AAl?$AAe?$AAU?$AAI?$AAE?$AAx?$AAt?$AA?$AA@ 00117ab8     Utilities.obj
 0002:00005ad4       ??_C@_1DO@GLFFNOLD@?$AAS?$AAO?$AAF?$AAT?$AAW?$AAA?$AAR?$AAE?$AA?2?$AAM?$AAi?$AAc?$AAr?$AAo?$AAs?$AAo?$AAf?$AAt?$AA?2?$AAS?$AAh?$AAe?$AAl?$AAl?$AA?2?$AAP?$AAh?$AAo?$AAn?$AAe?$AA?$AA@ 00117ad4     Utilities.obj
 0002:00005b14       ??_C@_1BM@CBFEBOB@?$AAG?$AAr?$AAo?$AAu?$AAp?$AAB?$AAr?$AAa?$AAn?$AAd?$AAi?$AAn?$AAg?$AA?$AA@ 00117b14     Utilities.obj
 0002:00005b30       ??_C@_15FPHCHCFA@?$AA?$CF?$AAi?$AA?$AA@ 00117b30     Utilities.obj
 0002:00005b38       ??_C@_1CE@JNKGAENM@?$AAF?$AAe?$AAa?$AAt?$AAu?$AAr?$AAe?$AAs?$AAS?$AAu?$AAp?$AAp?$AAo?$AAr?$AAt?$AAe?$AAd?$AA?$AA@ 00117b38     Utilities.obj
 0002:00005b60       ??_C@_1HC@GHOIHGLL@?$AAA?$AAd?$AAd?$AA?5?$AAD?$AAM?$AAP?$AAr?$AAo?$AAc?$AAe?$AAs?$AAs?$AAC?$AAo?$AAn?$AAf?$AAi?$AAg?$AAX?$AAM?$AAL?$AA?5?$AAf?$AAo?$AAr?$AA?5?$AAS?$AAW?$AAI?$AA?5?$AAP@ 00117b60     Utilities.obj
 0002:00005bd8       ??_C@_1GG@KMAKOIDC@?$AAA?$AAd?$AAd?$AA?5?$AAD?$AAM?$AAP?$AAr?$AAo?$AAc?$AAe?$AAs?$AAs?$AAC?$AAo?$AAn?$AAf?$AAi?$AAg?$AAX?$AAM?$AAL?$AA?5?$AAf?$AAo?$AAr?$AA?5?$AAP?$AAC?$AAS?$AA?5?$AAr@ 00117bd8     Utilities.obj
 0002:00005c40       ??_C@_1DA@IEDJCPCG@?$AAC?$AAA?$AAR?$AAR?$AAI?$AAE?$AAR?$AA?5?$AAI?$AAN?$AAD?$AAE?$AAX?$AA?5?$AAI?$AAS?$AA?5?$AAS?$AAP?$AAR?$AAI?$AAN?$AAT?$AA?$AA@ 00117c40     Utilities.obj
 0002:00005c70       ??_C@_1BG@JFIMKLMC@?$AAR?$AAe?$AAt?$AAr?$AAy?$AAC?$AAo?$AAu?$AAn?$AAt?$AA?$AA@ 00117c70     Utilities.obj
 0002:00005c88       ??_C@_1DO@FOHJJKMN@?$AAC?$AAo?$AAm?$AAm?$AA?2?$AAC?$AAo?$AAn?$AAn?$AAM?$AAg?$AAr?$AA?2?$AAP?$AAl?$AAa?$AAn?$AAn?$AAe?$AAr?$AA?2?$AAS?$AAe?$AAt?$AAt?$AAi?$AAn?$AAg?$AAs?$AA?2?$AA?$AA@ 00117c88     Utilities.obj
 0002:00005cc8       ??_C@_1GG@CPDEIIMP@?$AAA?$AAd?$AAd?$AA?5?$AAD?$AAM?$AAP?$AAr?$AAo?$AAc?$AAe?$AAs?$AAs?$AAC?$AAo?$AAn?$AAf?$AAi?$AAg?$AAX?$AAM?$AAL?$AA?5?$AAf?$AAo?$AAr?$AA?5?$AAV?$AAZ?$AAW?$AA?5?$AAr@ 00117cc8     Utilities.obj
 0002:00005d30       ??_C@_1DC@BKGMFHNE@?$AAC?$AAA?$AAR?$AAR?$AAI?$AAE?$AAR?$AA?5?$AAI?$AAN?$AAD?$AAE?$AAX?$AA?5?$AAI?$AAS?$AA?5?$AAV?$AAE?$AAR?$AAI?$AAZ?$AAO?$AAN?$AA?$AA@ 00117d30     Utilities.obj
 0002:00005d68       ??_C@_1GG@FJGONHKO@?$AAA?$AAd?$AAd?$AA?5?$AAD?$AAM?$AAP?$AAr?$AAo?$AAc?$AAe?$AAs?$AAs?$AAC?$AAo?$AAn?$AAf?$AAi?$AAg?$AAX?$AAM?$AAL?$AA?5?$AAf?$AAo?$AAr?$AA?5?$AAG?$AAS?$AAM?$AA?5?$AAr@ 00117d68     Utilities.obj
 0002:00005dd0       ??_C@_1CK@NDBPKJHI@?$AAC?$AAA?$AAR?$AAR?$AAI?$AAE?$AAR?$AA?5?$AAI?$AAN?$AAD?$AAE?$AAX?$AA?5?$AAI?$AAS?$AA?5?$AAG?$AAS?$AAM?$AA?$AA@ 00117dd0     Utilities.obj
 0002:00005e00       ??_C@_1IE@PLDBDLAC@?$AAR?$AAe?$AAm?$AAo?$AAv?$AAe?$AA?5?$AAD?$AAM?$AAP?$AAr?$AAo?$AAc?$AAe?$AAs?$AAs?$AAC?$AAo?$AAn?$AAf?$AAi?$AAg?$AAX?$AAM?$AAL?$AA?5?$AAf?$AAo?$AAr?$AA?5?$AAG?$AAS@ 00117e00     Utilities.obj
 0002:00005e84       ??_C@_1DM@JNJOFOLN@?$AAR?$AAE?$AAM?$AAO?$AAV?$AAI?$AAN?$AAG?$AA?5?$AAG?$AAS?$AAM?$AA?5?$AAC?$AAO?$AAN?$AAN?$AAE?$AAC?$AAT?$AAI?$AAO?$AAN?$AA?5?$AAE?$AAN?$AAT?$AAR?$AAY?$AA?$AA@ 00117e84     Utilities.obj
 0002:00005ec0       ??_C@_1JM@IKHPMDJP@?$AAR?$AAe?$AAm?$AAo?$AAv?$AAe?$AA?5?$AAD?$AAM?$AAP?$AAr?$AAo?$AAc?$AAe?$AAs?$AAs?$AAC?$AAo?$AAn?$AAf?$AAi?$AAg?$AAX?$AAM?$AAL?$AA?5?$AAf?$AAo?$AAr?$AA?5?$AAN?$AAa@ 00117ec0     Utilities.obj
 0002:00005f5c       ??_C@_1DO@BHCFBKNF@?$AAR?$AAE?$AAM?$AAO?$AAV?$AAI?$AAN?$AAG?$AA?5?$AAN?$AAA?$AAT?$AAI?$AAO?$AAN?$AAA?$AAL?$AA?5?$AAA?$AAC?$AAC?$AAE?$AAS?$AAS?$AA?5?$AAE?$AAN?$AAT?$AAR?$AAY?$AA?$AA@ 00117f5c     Utilities.obj
 0002:00005fa0       ??_C@_1IE@IOFCAAKP@?$AAR?$AAe?$AAm?$AAo?$AAv?$AAe?$AA?5?$AAD?$AAM?$AAP?$AAr?$AAo?$AAc?$AAe?$AAs?$AAs?$AAC?$AAo?$AAn?$AAf?$AAi?$AAg?$AAX?$AAM?$AAL?$AA?5?$AAf?$AAo?$AAr?$AA?5?$AAP?$AAC@ 00117fa0     Utilities.obj
 0002:00006024       ??_C@_1DE@PDAOJOCL@?$AAR?$AAE?$AAM?$AAO?$AAV?$AAI?$AAN?$AAG?$AA?5?$AAP?$AAC?$AAS?$AA?5?$AAV?$AAI?$AAS?$AAI?$AAO?$AAN?$AA?5?$AAE?$AAN?$AAT?$AAR?$AAY?$AA?$AA@ 00118024     Utilities.obj
 0002:00006058       ??_C@_1HA@JEHFMHKK@?$AAD?$AAo?$AAn?$AA?8?$AAt?$AA?5?$AAk?$AAn?$AAo?$AAw?$AA?5?$AAt?$AAo?$AA?5?$AAh?$AAa?$AAn?$AAd?$AAl?$AAe?$AA?5?$AAs?$AAz?$AAB?$AAu?$AAf?$AAf?$AAe?$AAr?$AA?5?$AA?$DN?$AA?5@ 00118058     Utilities.obj
 0002:000060c8       ??_C@_1HE@BIONCIBO@?$AAC?$AAA?$AAR?$AAR?$AAI?$AAE?$AAR?$AA?5?$AAI?$AAN?$AAD?$AAE?$AAX?$AA?5?$AAW?$AAA?$AAS?$AA?5?$AAG?$AAS?$AAM?$AA?0?$AA?5?$AAs?$AAz?$AAB?$AAu?$AAf?$AAf?$AAe?$AAr?$AA?5@ 001180c8     Utilities.obj
 0002:0000613c       ??_C@_1BO@IGCNNIBP@?$AAG?$AAS?$AAM?$AA?5?$AAC?$AAo?$AAn?$AAn?$AAe?$AAc?$AAt?$AAi?$AAo?$AAn?$AA?$AA@ 0011813c     Utilities.obj
 0002:0000615c       ??_C@_1CA@IEFLIGMG@?$AA?4?$AA?2?$AAU?$AAt?$AAi?$AAl?$AAi?$AAt?$AAi?$AAe?$AAs?$AA?4?$AAc?$AAp?$AAp?$AA?$AA@ 0011815c     Utilities.obj
 0002:00006180       ??_C@_1HM@IOJOEMIG@?$AAC?$AAA?$AAR?$AAR?$AAI?$AAE?$AAR?$AA?5?$AAI?$AAN?$AAD?$AAE?$AAX?$AA?5?$AAW?$AAA?$AAS?$AA?5?$AAV?$AAE?$AAR?$AAI?$AAZ?$AAO?$AAN?$AA?0?$AA?5?$AAs?$AAz?$AAB?$AAu?$AAf@ 00118180     Utilities.obj
 0002:000061fc       ??_C@_1BO@KHEAMGKD@?$AAN?$AAa?$AAt?$AAi?$AAo?$AAn?$AAa?$AAl?$AAA?$AAc?$AAc?$AAe?$AAs?$AAs?$AA?$AA@ 001181fc     Utilities.obj
 0002:0000621c       ??_C@_1BG@FNBKCOCE@?$AAP?$AAC?$AAS?$AA?5?$AAV?$AAi?$AAs?$AAi?$AAo?$AAn?$AA?$AA@ 0011821c     Utilities.obj
 0002:00006234       ??_C@_1DE@JKKCOFKH@?$AAC?$AAo?$AAm?$AAm?$AA?2?$AAC?$AAo?$AAn?$AAn?$AAM?$AAg?$AAr?$AA?2?$AAD?$AAe?$AAs?$AAt?$AAi?$AAn?$AAa?$AAt?$AAi?$AAo?$AAn?$AAs?$AA?$AA@ 00118234     Utilities.obj
 0002:00006268       ??_C@_1CG@LCGGEEDP@?$AAD?$AAM?$AAP?$AAr?$AAo?$AAc?$AAe?$AAs?$AAs?$AAC?$AAo?$AAn?$AAf?$AAi?$AAg?$AAX?$AAM?$AAL?$AA?$AA@ 00118268     Utilities.obj
 0002:00006290       ??_C@_1BK@HMCKJION@?$AAa?$AAy?$AAg?$AAs?$AAh?$AAe?$AAl?$AAl?$AA?4?$AAd?$AAl?$AAl?$AA?$AA@ 00118290     Utilities.obj
 0002:000062b0       ??_C@_1IE@OBJAMJDB@?$AAU?$AAn?$AAa?$AAb?$AAl?$AAe?$AA?5?$AAt?$AAo?$AA?5?$AAo?$AAp?$AAe?$AAn?$AA?5?$AAt?$AAh?$AAe?$AA?5?$AAr?$AAe?$AAg?$AAi?$AAs?$AAt?$AAr?$AAy?$AA?5?$AAk?$AAe?$AAy?$AA?5@ 001182b0     Utilities.obj
 0002:00006338       ??_C@_1FM@JFNCIKHA@?$AAU?$AAn?$AAa?$AAb?$AAl?$AAe?$AA?5?$AAS?$AAe?$AAt?$AA?5?$AAF?$AAe?$AAa?$AAt?$AAu?$AAr?$AAe?$AAs?$AA?5?$AAw?$AAi?$AAt?$AAh?$AA?5?$AAv?$AAa?$AAl?$AAu?$AAe?$AA?5?$AA?$CF@ 00118338     Utilities.obj
 0002:00006398       ??_C@_1EE@GJFHCOH@?$AAU?$AAn?$AAa?$AAb?$AAl?$AAe?$AA?5?$AAQ?$AAu?$AAe?$AAr?$AAy?$AA?5?$AAF?$AAe?$AAa?$AAt?$AAu?$AAr?$AAe?$AAs?$AA?5?$AA?5?$AAe?$AAr?$AAr?$AAo?$AAr?$AA?5?$AA?$DN?$AA?5?$AA?$CF@ 00118398     Utilities.obj
 0002:000063dc       ??_C@_1BC@IGDFDBLI@?$AAF?$AAe?$AAa?$AAt?$AAu?$AAr?$AAe?$AAs?$AA?$AA@ 001183dc     Utilities.obj
 0002:000063f0       ??_C@_1CG@LJBEDMCE@?$AAC?$AAo?$AAn?$AAt?$AAr?$AAo?$AAl?$AAP?$AAa?$AAn?$AAe?$AAl?$AA?2?$AAP?$AAh?$AAo?$AAn?$AAe?$AA?$AA@ 001183f0     Utilities.obj
 0002:00006418       ??_C@_1KI@DICDMDEI@?$AAU?$AAn?$AAa?$AAb?$AAl?$AAe?$AA?5?$AAt?$AAo?$AA?5?$AAo?$AAp?$AAe?$AAn?$AA?1?$AAc?$AAr?$AAe?$AAa?$AAt?$AAe?$AA?5?$AAt?$AAh?$AAe?$AA?5?$AAr?$AAe?$AAg?$AAi?$AAs?$AAt@ 00118418     Utilities.obj
 0002:000064c0       ??_C@_1IG@FOFNBLON@?$AAU?$AAn?$AAa?$AAb?$AAl?$AAe?$AA?5?$AAt?$AAo?$AA?5?$AAs?$AAe?$AAt?$AA?5?$AAt?$AAh?$AAe?$AA?5?$AAB?$AAa?$AAs?$AAe?$AAD?$AAl?$AAl?$AA?5?$AAH?$AAK?$AAL?$AAM?$AA?2?$AAS@ 001184c0     Utilities.obj
 0002:00006548       ??_C@_1IE@KBDPABC@?$AAU?$AAn?$AAa?$AAb?$AAl?$AAe?$AA?5?$AAt?$AAo?$AA?5?$AAs?$AAe?$AAt?$AA?5?$AAt?$AAh?$AAe?$AA?5?$AAB?$AAa?$AAs?$AAe?$AAI?$AAd?$AA?5?$AAH?$AAK?$AAL?$AAM?$AA?2?$AAS?$AAe@ 00118548     Utilities.obj
 0002:000065d0       ??_C@_1JK@JLMPHBPL@?$AAU?$AAn?$AAa?$AAb?$AAl?$AAe?$AA?5?$AAt?$AAo?$AA?5?$AAo?$AAp?$AAe?$AAn?$AA?5?$AAt?$AAh?$AAe?$AA?5?$AAr?$AAe?$AAg?$AAi?$AAs?$AAt?$AAr?$AAy?$AA?5?$AAk?$AAe?$AAy?$AA?5@ 001185d0     Utilities.obj
 0002:00006670       ??_C@_1IM@LHNKNIAA@?$AAU?$AAn?$AAa?$AAb?$AAl?$AAe?$AA?5?$AAt?$AAo?$AA?5?$AAd?$AAe?$AAl?$AAe?$AAt?$AAe?$AA?5?$AAt?$AAh?$AAe?$AA?5?$AAB?$AAa?$AAs?$AAe?$AAD?$AAl?$AAl?$AA?5?$AAH?$AAK?$AAL@ 00118670     Utilities.obj
 0002:000066fc       ??_C@_1BA@GMEDNONB@?$AAB?$AAa?$AAs?$AAe?$AAD?$AAl?$AAl?$AA?$AA@ 001186fc     Utilities.obj
 0002:00006710       ??_C@_1IK@GCAEPNJO@?$AAU?$AAn?$AAa?$AAb?$AAl?$AAe?$AA?5?$AAt?$AAo?$AA?5?$AAd?$AAe?$AAl?$AAe?$AAt?$AAe?$AA?5?$AAt?$AAh?$AAe?$AA?5?$AAB?$AAa?$AAs?$AAe?$AAI?$AAd?$AA?5?$AAH?$AAK?$AAL?$AAM@ 00118710     Utilities.obj
 0002:0000679c       ??_C@_1O@CEACDOLH@?$AAB?$AAa?$AAs?$AAe?$AAI?$AAd?$AA?$AA@ 0011879c     Utilities.obj
 0002:000067ac       ??_C@_1DC@ODCINLCC@?$AAS?$AAe?$AAc?$AAu?$AAr?$AAi?$AAt?$AAy?$AA?2?$AAR?$AAe?$AAs?$AAO?$AAv?$AAe?$AAr?$AA?2?$AAB?$AAi?$AAt?$AAm?$AAa?$AAp?$AAs?$AA?$AA@ 001187ac     Utilities.obj
 0002:000067e0       ??_C@_1BO@NEMDOCHC@?$AAs?$AAw?$AAi?$AA_?$AAr?$AAi?$AAl?$AAr?$AAe?$AAs?$AA?4?$AAd?$AAl?$AAl?$AA?$AA@ 001187e0     Utilities.obj
 0002:00006800       ??_C@_1GE@IDHCHKIP@?$AAS?$AAp?$AAe?$AAi?$AAc?$AAi?$AAa?$AAl?$AA?5?$AAN?$AAu?$AAm?$AAb?$AAe?$AAr?$AA?5?$AAi?$AAs?$AA?5?$AAs?$AAe?$AAt?$AA?3?$AA?5?$AAR?$AAe?$AAg?$AAi?$AAs?$AAt?$AAr?$AAy@ 00118800     Utilities.obj
 0002:00006868       ??_C@_1GO@MEKNLFCF@?$AAU?$AAn?$AAa?$AAb?$AAl?$AAe?$AA?5?$AAt?$AAo?$AA?5?$AAs?$AAe?$AAt?$AA?5?$AAR?$AAe?$AAg?$AAi?$AAs?$AAt?$AAr?$AAy?$AA?5?$AA?$CF?$AAs?$AA?5?$AAf?$AAo?$AAr?$AA?5?$AAs?$AAp@ 00118868     Utilities.obj
 0002:000068d8       ??_C@_1BM@PJPNMBMC@?$AAS?$AAp?$AAe?$AAc?$AAi?$AAa?$AAl?$AAN?$AAu?$AAm?$AAb?$AAe?$AAr?$AA?$AA@ 001188d8     Utilities.obj
 0002:000068f8       ??_C@_1FO@GHPCFLAO@?$AAS?$AAp?$AAe?$AAi?$AAc?$AAi?$AAa?$AAl?$AA?5?$AAN?$AAu?$AAm?$AAb?$AAe?$AAr?$AA?5?$AAi?$AAs?$AA?5?$AA?3?$AA?5?$AAR?$AAe?$AAg?$AAi?$AAs?$AAt?$AAr?$AAy?$AA?5?$AA?$CF?$AAs@ 001188f8     Utilities.obj
 0002:00006958       ??_C@_1EC@OJBKIBEO@?$AAU?$AAn?$AAa?$AAb?$AAl?$AAe?$AA?5?$AAt?$AAo?$AA?5?$AAg?$AAe?$AAt?$AA?5?$AAR?$AAe?$AAg?$AAi?$AAs?$AAt?$AAr?$AAy?$AA?5?$AA?$CF?$AAs?$AA?5?$AAE?$AAr?$AAr?$AA?5?$AA?$CF?$AAd@ 00118958     Utilities.obj
 0002:0000699c       ??_C@_1BA@OJFOBGOM@?$AA0?$AA?4?$AA0?$AA?4?$AA0?$AA?4?$AA0?$AA?$AA@ 0011899c     Utilities.obj
 0002:000069ac       ??_C@_1BI@KONPHAJJ@?$AA?$CF?$AAi?$AA?4?$AA?$CF?$AAi?$AA?4?$AA?$CF?$AAi?$AA?4?$AA?$CF?$AAi?$AA?$AA@ 001189ac     Utilities.obj
 0002:000069c8       ??_C@_1II@JMIEAIHF@?$AAU?$AAn?$AAa?$AAb?$AAl?$AAe?$AA?5?$AAt?$AAo?$AA?5?$AAs?$AAe?$AAt?$AA?5?$AAR?$AAe?$AAg?$AAi?$AAs?$AAt?$AAr?$AAy?$AA?5?$AA?$CF?$AAs?$AA?5?$AAf?$AAo?$AAr?$AA?5?$AAc?$AAa@ 001189c8     Utilities.obj
 0002:00006a50       ??_C@_1CM@PGIJNMC@?$AAC?$AAo?$AAn?$AAn?$AAe?$AAc?$AAt?$AAi?$AAo?$AAn?$AAP?$AAr?$AAo?$AAf?$AAi?$AAl?$AAe?$AAN?$AAa?$AAm?$AAe?$AA?$AA@ 00118a50     Utilities.obj
 0002:00006a80       ??_C@_1II@FBOAHAKN@?$AAU?$AAn?$AAa?$AAb?$AAl?$AAe?$AA?5?$AAt?$AAo?$AA?5?$AAs?$AAe?$AAt?$AA?5?$AAR?$AAe?$AAg?$AAi?$AAs?$AAt?$AAr?$AAy?$AA?5?$AA?$CF?$AAs?$AA?5?$AAf?$AAo?$AAr?$AA?5?$AAc?$AAa@ 00118a80     Utilities.obj
 0002:00006b08       ??_C@_1BM@LABJEMAB@?$AA3?$AAG?$AA?5?$AAC?$AAo?$AAn?$AAn?$AAe?$AAc?$AAt?$AAi?$AAo?$AAn?$AA?$AA@ 00118b08     Utilities.obj
 0002:00006b24       ??_C@_1BA@HDEOAKLJ@?$AAT?$AAe?$AAl?$AAe?$AAc?$AAo?$AAm?$AA?$AA@ 00118b24     Utilities.obj
 0002:00006b34       ??_C@_1BE@MKENKGHK@?$AAR?$AAU?$AAI?$AAM?$AA?5?$AAC?$AAD?$AAM?$AAA?$AA?$AA@ 00118b34     Utilities.obj
 0002:00006b48       ??_C@_1GA@FEGEOOFM@?$AAC?$AAa?$AAr?$AAr?$AAi?$AAe?$AAr?$AAI?$AAn?$AAd?$AAe?$AAx?$AAc?$AAh?$AAa?$AAn?$AAg?$AAe?$AAd?$AA?5?$AAo?$AAl?$AAd?$AAC?$AAa?$AAr?$AAr?$AAi?$AAe?$AAr?$AA?5?$AA?$CF@ 00118b48     Utilities.obj
 0002:00006ba8       ??_C@_13JOFGPIOO@?$AA?4?$AA?$AA@ 00118ba8     Utilities.obj
 0002:00006bac       GUID_ATLVer30              00118bac     atls:atlbase.obj
 0002:00006bbc       GUID_ATLVer70              00118bbc     atls:atlbase.obj
 0002:00006bcc       IID_IPersistStream         00118bcc     uuid:objidl_i_guid12.obj
 0002:00006cc0       __IMPORT_DESCRIPTOR_COREDLL 00118cc0     coredll:COREDLL.dll
 0002:00006cd4       __IMPORT_DESCRIPTOR_ril    00118cd4     ril:ril.dll
 0002:00006ce8       __IMPORT_DESCRIPTOR_WS2    00118ce8     ws2:WS2.dll
 0002:00006cfc       __NULL_IMPORT_DESCRIPTOR   00118cfc     coredll:COREDLL.dll
 0003:00000000       __imp_memcpy               0011b000     coredll:COREDLL.dll
 0003:00000004       __imp_??3@YAXPAX@Z         0011b004     coredll:COREDLL.dll
 0003:00000008       __imp_GetFileVersionInfoW  0011b008     coredll:COREDLL.dll
 0003:0000000c       __imp_??2@YAPAXI@Z         0011b00c     coredll:COREDLL.dll
 0003:00000010       __imp_GetFileVersionInfoSizeW 0011b010     coredll:COREDLL.dll
 0003:00000014       __imp_wcscpy               0011b014     coredll:COREDLL.dll
 0003:00000018       __imp_OutputDebugStringW   0011b018     coredll:COREDLL.dll
 0003:0000001c       __imp_swprintf             0011b01c     coredll:COREDLL.dll
 0003:00000020       __imp_VerQueryValueW       0011b020     coredll:COREDLL.dll
 0003:00000024       __imp_wcscat               0011b024     coredll:COREDLL.dll
 0003:00000028       __imp_GetModuleFileNameW   0011b028     coredll:COREDLL.dll
 0003:0000002c       __imp_EventModify          0011b02c     coredll:COREDLL.dll
 0003:00000030       __imp_InitializeCriticalSection 0011b030     coredll:COREDLL.dll
 0003:00000034       __imp_DeleteCriticalSection 0011b034     coredll:COREDLL.dll
 0003:00000038       __imp_EnterCriticalSection 0011b038     coredll:COREDLL.dll
 0003:0000003c       __imp_LeaveCriticalSection 0011b03c     coredll:COREDLL.dll
 0003:00000040       __imp_RegisterWindowMessageW 0011b040     coredll:COREDLL.dll
 0003:00000044       __imp_CreateEventW         0011b044     coredll:COREDLL.dll
 0003:00000048       __imp_wsprintfW            0011b048     coredll:COREDLL.dll
 0003:0000004c       __imp_WaitForSingleObject  0011b04c     coredll:COREDLL.dll
 0003:00000050       __imp_memset               0011b050     coredll:COREDLL.dll
 0003:00000054       __imp_PostMessageW         0011b054     coredll:COREDLL.dll
 0003:00000058       __imp_CloseHandle          0011b058     coredll:COREDLL.dll
 0003:0000005c       __imp_CreateThread         0011b05c     coredll:COREDLL.dll
 0003:00000060       __imp_wcslen               0011b060     coredll:COREDLL.dll
 0003:00000064       __imp_strcpy               0011b064     coredll:COREDLL.dll
 0003:00000068       __imp_wcsncpy              0011b068     coredll:COREDLL.dll
 0003:0000006c       __imp_strlen               0011b06c     coredll:COREDLL.dll
 0003:00000070       __imp___C_specific_handler 0011b070     coredll:COREDLL.dll
 0003:00000074       __imp_free                 0011b074     coredll:COREDLL.dll
 0003:00000078       __imp_CloseMsgQueue        0011b078     coredll:COREDLL.dll
 0003:0000007c       __imp_TerminateThread      0011b07c     coredll:COREDLL.dll
 0003:00000080       __imp_WriteMsgQueue        0011b080     coredll:COREDLL.dll
 0003:00000084       __imp_PurgeComm            0011b084     coredll:COREDLL.dll
 0003:00000088       __imp_SetCommMask          0011b088     coredll:COREDLL.dll
 0003:0000008c       __imp_SetCommTimeouts      0011b08c     coredll:COREDLL.dll
 0003:00000090       __imp_SetCommState         0011b090     coredll:COREDLL.dll
 0003:00000094       __imp_GetCommState         0011b094     coredll:COREDLL.dll
 0003:00000098       __imp_MessageBoxW          0011b098     coredll:COREDLL.dll
 0003:0000009c       __imp_wcsstr               0011b09c     coredll:COREDLL.dll
 0003:000000a0       __imp__wcslwr              0011b0a0     coredll:COREDLL.dll
 0003:000000a4       __imp_DeleteFileW          0011b0a4     coredll:COREDLL.dll
 0003:000000a8       __imp_FlushFileBuffers     0011b0a8     coredll:COREDLL.dll
 0003:000000ac       __imp_WriteFile            0011b0ac     coredll:COREDLL.dll
 0003:000000b0       __imp_GetLastError         0011b0b0     coredll:COREDLL.dll
 0003:000000b4       __imp_CreateFileW          0011b0b4     coredll:COREDLL.dll
 0003:000000b8       __imp_CopyFileW            0011b0b8     coredll:COREDLL.dll
 0003:000000bc       __imp_GetFileSize          0011b0bc     coredll:COREDLL.dll
 0003:000000c0       __imp_Sleep                0011b0c0     coredll:COREDLL.dll
 0003:000000c4       __imp_NKDbgPrintfW         0011b0c4     coredll:COREDLL.dll
 0003:000000c8       __imp_GetLocalTime         0011b0c8     coredll:COREDLL.dll
 0003:000000cc       __imp_vswprintf            0011b0cc     coredll:COREDLL.dll
 0003:000000d0       __imp_wcscmp               0011b0d0     coredll:COREDLL.dll
 0003:000000d4       __imp_ReadMsgQueue         0011b0d4     coredll:COREDLL.dll
 0003:000000d8       __imp_CreateMsgQueue       0011b0d8     coredll:COREDLL.dll
 0003:000000dc       __imp_SetFilePointer       0011b0dc     coredll:COREDLL.dll
 0003:000000e0       __imp_ReleaseMutex         0011b0e0     coredll:COREDLL.dll
 0003:000000e4       __imp_CreateMutexW         0011b0e4     coredll:COREDLL.dll
 0003:000000e8       __imp_GetStoreInformation  0011b0e8     coredll:COREDLL.dll
 0003:000000ec       __imp_GlobalMemoryStatus   0011b0ec     coredll:COREDLL.dll
 0003:000000f0       __imp_rand                 0011b0f0     coredll:COREDLL.dll
 0003:000000f4       __imp_RegDeleteKeyW        0011b0f4     coredll:COREDLL.dll
 0003:000000f8       __imp_RegOpenKeyExW        0011b0f8     coredll:COREDLL.dll
 0003:000000fc       __imp_RegCloseKey          0011b0fc     coredll:COREDLL.dll
 0003:00000100       __imp_RegQueryValueExW     0011b100     coredll:COREDLL.dll
 0003:00000104       __imp_RegSetValueExW       0011b104     coredll:COREDLL.dll
 0003:00000108       __imp_RegEnumKeyExW        0011b108     coredll:COREDLL.dll
 0003:0000010c       __imp_wcschr               0011b10c     coredll:COREDLL.dll
 0003:00000110       __imp_RegCreateKeyExW      0011b110     coredll:COREDLL.dll
 0003:00000114       __imp_RegEnumValueW        0011b114     coredll:COREDLL.dll
 0003:00000118       __imp_GetVersionExW        0011b118     coredll:COREDLL.dll
 0003:0000011c       __imp__wcsicmp             0011b11c     coredll:COREDLL.dll
 0003:00000120       __imp__wtol                0011b120     coredll:COREDLL.dll
 0003:00000124       __imp_mbstowcs             0011b124     coredll:COREDLL.dll
 0003:00000128       __imp_wcstombs             0011b128     coredll:COREDLL.dll
 0003:0000012c       __imp_SetDlgItemTextW      0011b12c     coredll:COREDLL.dll
 0003:00000130       __imp_DeleteObject         0011b130     coredll:COREDLL.dll
 0003:00000134       __imp_LoadBitmapW          0011b134     coredll:COREDLL.dll
 0003:00000138       __imp_DestroyIcon          0011b138     coredll:COREDLL.dll
 0003:0000013c       __imp_LoadIconW            0011b13c     coredll:COREDLL.dll
 0003:00000140       __imp_SendDlgItemMessageW  0011b140     coredll:COREDLL.dll
 0003:00000144       __imp_GetSystemMetrics     0011b144     coredll:COREDLL.dll
 0003:00000148       __imp_SendMessageW         0011b148     coredll:COREDLL.dll
 0003:0000014c       __imp_FreeLibrary          0011b14c     coredll:COREDLL.dll
 0003:00000150       __imp_GetProcAddressW      0011b150     coredll:COREDLL.dll
 0003:00000154       __imp_LoadLibraryW         0011b154     coredll:COREDLL.dll
 0003:00000158       __imp_RegDeleteValueW      0011b158     coredll:COREDLL.dll
 0003:0000015c       __imp_SetCursor            0011b15c     coredll:COREDLL.dll
 0003:00000160       __imp_LoadCursorW          0011b160     coredll:COREDLL.dll
 0003:00000164       __imp_FileTimeToSystemTime 0011b164     coredll:COREDLL.dll
 0003:00000168       __imp_LocalFileTimeToFileTime 0011b168     coredll:COREDLL.dll
 0003:0000016c       __imp_SystemTimeToFileTime 0011b16c     coredll:COREDLL.dll
 0003:00000170       __imp_EndDeferWindowPos    0011b170     coredll:COREDLL.dll
 0003:00000174       __imp_DeferWindowPos       0011b174     coredll:COREDLL.dll
 0003:00000178       __imp_MapDialogRect        0011b178     coredll:COREDLL.dll
 0003:0000017c       __imp_GetDlgItem           0011b17c     coredll:COREDLL.dll
 0003:00000180       __imp_BeginDeferWindowPos  0011b180     coredll:COREDLL.dll
 0003:00000184       __imp_LoadResource         0011b184     coredll:COREDLL.dll
 0003:00000188       __imp_FindResourceW        0011b188     coredll:COREDLL.dll
 0003:0000018c       __imp_InterlockedCompareExchange 0011b18c     coredll:COREDLL.dll
 0003:00000190       __imp_TlsGetValue          0011b190     coredll:COREDLL.dll
 0003:00000194       __imp_TlsSetValue          0011b194     coredll:COREDLL.dll
 0003:00000198       __imp_TlsCall              0011b198     coredll:COREDLL.dll
 0003:0000019c       __imp_memmove              0011b19c     coredll:COREDLL.dll
 0003:000001a0       __imp_?terminate@std@@YAXXZ 0011b1a0     coredll:COREDLL.dll
 0003:000001a4       __imp_strcmp               0011b1a4     coredll:COREDLL.dll
 0003:000001a8       __imp_GetModuleHandleW     0011b1a8     coredll:COREDLL.dll
 0003:000001ac       __imp___security_gen_cookie 0011b1ac     coredll:COREDLL.dll
 0003:000001b0       __imp_DisableThreadLibraryCalls 0011b1b0     coredll:COREDLL.dll
 0003:000001b4       __imp_LocalFree            0011b1b4     coredll:COREDLL.dll
 0003:000001b8       __imp_LocalSize            0011b1b8     coredll:COREDLL.dll
 0003:000001bc       __imp_LocalAlloc           0011b1bc     coredll:COREDLL.dll
 0003:000001c0       __imp_LocalReAlloc         0011b1c0     coredll:COREDLL.dll
 0003:000001c4       __imp___report_gsfailure   0011b1c4     coredll:COREDLL.dll
 0003:000001c8       \177COREDLL_NULL_THUNK_DATA 0011b1c8     coredll:COREDLL.dll
 0003:000001cc       __imp_ntohl                0011b1cc     ws2:WS2.dll
 0003:000001d0       \177WS2_NULL_THUNK_DATA    0011b1d0     ws2:WS2.dll
 0003:000001d4       __imp_RIL_SetRoamingMode   0011b1d4     ril:ril.dll
 0003:000001d8       __imp_RIL_GetRoamingMode   0011b1d8     ril:ril.dll
 0003:000001dc       __imp_RIL_GetPreferredPrivacyMode 0011b1dc     ril:ril.dll
 0003:000001e0       __imp_RIL_Dial             0011b1e0     ril:ril.dll
 0003:000001e4       __imp_RIL_Hangup           0011b1e4     ril:ril.dll
 0003:000001e8       __imp_RIL_SetEquipmentState 0011b1e8     ril:ril.dll
 0003:000001ec       __imp_RIL_SetPreferredPrivacyMode 0011b1ec     ril:ril.dll
 0003:000001f0       __imp_RIL_Initialize       0011b1f0     ril:ril.dll
 0003:000001f4       __imp_RIL_GetCallList      0011b1f4     ril:ril.dll
 0003:000001f8       __imp_RIL_GetCurrentSystemType 0011b1f8     ril:ril.dll
 0003:000001fc       __imp_RIL_GetRegistrationStatus 0011b1fc     ril:ril.dll
 0003:00000200       __imp_RIL_GetEquipmentState 0011b200     ril:ril.dll
 0003:00000204       __imp_RIL_DevSpecific      0011b204     ril:ril.dll
 0003:00000208       __imp_RIL_Deinitialize     0011b208     ril:ril.dll
 0003:0000020c       __imp_RIL_GetPacketByteCount 0011b20c     ril:ril.dll
 0003:00000210       __imp_RIL_GetUserIdentity  0011b210     ril:ril.dll
 0003:00000214       __imp_RIL_SendAKey         0011b214     ril:ril.dll
 0003:00000218       \177ril_NULL_THUNK_DATA    0011b218     ril:ril.dll
 0003:0000021c       __xc_a                     0011b21c     corelibc:crt0init.obj
 0003:00000238       __xc_z                     0011b238     corelibc:crt0init.obj
 0003:0000023c       __xi_a                     0011b23c     corelibc:crt0init.obj
 0003:00000240       __xi_z                     0011b240     corelibc:crt0init.obj
 0003:00000244       __xp_a                     0011b244     corelibc:crt0init.obj
 0003:00000248       __xp_z                     0011b248     corelibc:crt0init.obj
 0003:0000024c       __xt_a                     0011b24c     corelibc:crt0init.obj
 0003:00000250       __xt_z                     0011b250     corelibc:crt0init.obj
 0003:0000025c       ?gCommandCS@@3VCriticalSection@@A 0011b25c     ModemStat.obj
 0003:00000274       ?g_hLogOpenedBy1stApp@@3PAXA 0011b274     SW_Log.obj
 0003:00000278       ?theSWIDisplayRawDataCR@@3VCriticalSection@@A 0011b278     SW_Log_Include.obj
 0003:00000294       ?g_wszSetupSWIProxy@@3PBGB 0011b294     Utilities.obj
 0003:00000298       ?g_wszSetupGSMXml@@3PBGB   0011b298     Utilities.obj
 0003:0000029c       ?g_wszSetupPCSXml@@3PBGB   0011b29c     Utilities.obj
 0003:000002a0       ?g_wszSetupVZWXml@@3PBGB   0011b2a0     Utilities.obj
 0003:000002a4       ?g_wszRemoveGSMNetworkXml@@3PBGB 0011b2a4     Utilities.obj
 0003:000002a8       ?g_wszRemoveGSMEntriesXml@@3PBGB 0011b2a8     Utilities.obj
 0003:000002ac       ?g_wszRemovePCSNetworkXml@@3PBGB 0011b2ac     Utilities.obj
 0003:000002b0       ?g_wszRemovePCSEntriesXml@@3PBGB 0011b2b0     Utilities.obj
 0003:000002b4       ?g_wszRemoveVZWNetworkXml@@3PBGB 0011b2b4     Utilities.obj
 0003:000002b8       ?g_wszRemoveVZWEntriesXml@@3PBGB 0011b2b8     Utilities.obj
 0003:000002bc       __security_cookie_complement 0011b2bc     corelibc:seccook.obj
 0003:000002c0       __security_cookie          0011b2c0     corelibc:seccook.obj
 0003:000002c4       _pRawDllMain               0011b2c4     atls:atlbase.obj
 0003:000002d0       ?RIL_STATUS_CHANGED@CModemStatus@@2IA 0011b2d0     ModemStat.obj
 0003:000002d4       ?RIL_DBG_NOTIFY@CModemStatus@@2IA 0011b2d4     ModemStat.obj
 0003:000002d8       ?RIL_TECHHDR_NOTIFY@CModemStatus@@2IA 0011b2d8     ModemStat.obj
 0003:000002dc       ?RIL_IOTA_STATUS_CHANGED@CModemStatus@@2IA 0011b2dc     ModemStat.obj
 0003:000002e0       ?RIL_IOTA_WAP_URI@CModemStatus@@2IA 0011b2e0     ModemStat.obj
 0003:000002e4       ?RIL_PDSM_PD_DATA@CModemStatus@@2IA 0011b2e4     ModemStat.obj
 0003:000002e8       ?RIL_PDSM_PD_DONE@CModemStatus@@2IA 0011b2e8     ModemStat.obj
 0003:000002ec       ?RIL_PDSM_PD_END@CModemStatus@@2IA 0011b2ec     ModemStat.obj
 0003:000002f0       ?RIL_PDSM_PD_BEGIN@CModemStatus@@2IA 0011b2f0     ModemStat.obj
 0003:000002f4       ?RIL_PDSM_PD_UPDATE_FAILURE@CModemStatus@@2IA 0011b2f4     ModemStat.obj
 0003:000002f8       ?RIL_PDSM_PD_DLD_DATA@CModemStatus@@2IA 0011b2f8     ModemStat.obj
 0003:000002fc       ?RIL_PDSM_PD_DLD_DONE@CModemStatus@@2IA 0011b2fc     ModemStat.obj
 0003:00000300       ?RIL_PDSM_PD_DLD_END@CModemStatus@@2IA 0011b300     ModemStat.obj
 0003:00000304       ?RIL_PDSM_PD_DLD_BEGIN@CModemStatus@@2IA 0011b304     ModemStat.obj
 0003:00000308       ?RIL_PDSM_PA_PARAM@CModemStatus@@2IA 0011b308     ModemStat.obj
 0003:0000030c       ?RIL_CALL_BYTE_CTR@CModemStatus@@2IA 0011b30c     ModemStat.obj
 0003:00000310       ?g_objModemStatus@@3VCModemStatus@@A 0011b310     ModemStat.obj
 0003:000008b4       ?m_bInitFailed@CAtlBaseModule@ATL@@2_NA 0011b8b4     stdafx.obj
 0003:000008b8       ?m_msgBoxText@SW_Log@@0PAGA 0011b8b8     SW_Log.obj
 0003:00001ac8       ?g_MaxReachCount@@3KA      0011cac8     SW_Log.obj
 0003:00001ad0       ?g_Log@@3VSW_Log@@A        0011cad0     SW_Log.obj
 0003:00001d18       ?szOneLine@@3PAGA          0011cd18     SW_Log_Include.obj
 0003:00002518       ?g_nLine@@3HA              0011d518     SW_Log_Include.obj
 0003:00002520       ?g_szFile@@3PAGA           0011d520     SW_Log_Include.obj
 0003:00002728       ?strFormatVer@@3PAGA       0011d728     Utilities.obj
 0003:00002930       ?g_dwOSMajVer@@3KA         0011d930     Utilities.obj
 0003:00002b38       ?_pAtlRawDllMain@@3P6AHPAXK0@ZA 0011db38     atls:atlbase.obj
 0003:00002b3c       ?_AtlModuleInstance@ATL@@3PAUHINSTANCE__@@A 0011db3c     atls:atlbase.obj
 0003:00002b40       ?_AtlBaseModule@ATL@@3VCAtlBaseModule@1@A 0011db40     atls:atlbase.obj
 0003:00002b74       __onexitend                0011db74     <common>
 0003:00002b78       __onexitbegin              0011db78     <common>
 0003:00002b7c       _exitflag                  0011db7c     <common>

 entry point at        0001:0000ea0c

 Static symbols

 0001:00001528       __unwind$35592             00102528 f   ModemStat.obj
 0001:00001678       __unwind$35668             00102678 f   ModemStat.obj
 0001:000017c8       __unwind$35737             001027c8 f   ModemStat.obj
 0001:00001918       __unwind$35806             00102918 f   ModemStat.obj
 0001:00001a68       __unwind$35875             00102a68 f   ModemStat.obj
 0001:000036a0       __unwind$36852             001046a0 f   ModemStat.obj
 0001:00009d14       __unwind$46919             0010ad14 f   SW_Log_Include.obj
 0001:0000a704       __unwind$47778             0010b704 f   SW_Registrykey.obj
 0001:0000a71c       __unwind$47779             0010b71c f   SW_Registrykey.obj
 0001:0000a820       __unwind$47944             0010b820 f   SW_Registrykey.obj
 0001:0000a95c       __unwind$48074             0010b95c f   SW_Registrykey.obj
 0001:0000aa6c       __unwind$48198             0010ba6c f   SW_Registrykey.obj
 0001:0000ab34       __unwind$48320             0010bb34 f   SW_Registrykey.obj
 0001:0000ac0c       __unwind$48437             0010bc0c f   SW_Registrykey.obj
 0001:0000acd4       __unwind$48569             0010bcd4 f   SW_Registrykey.obj
 0001:0000ae18       __unwind$48687             0010be18 f   SW_Registrykey.obj
 0001:0000aff0       __unwind$48821             0010bff0 f   SW_Registrykey.obj
 0001:0000b1a4       __unwind$48957             0010c1a4 f   SW_Registrykey.obj
 0001:0000b2dc       __unwind$49091             0010c2dc f   SW_Registrykey.obj
 0001:0000b420       __unwind$49221             0010c420 f   SW_Registrykey.obj
 0001:0000b55c       __unwind$49366             0010c55c f   SW_Registrykey.obj
 0001:0000b7e8       __unwind$49496             0010c7e8 f   SW_Registrykey.obj
 0001:0000b808       __unwind$49497             0010c808 f   SW_Registrykey.obj
 0001:0000b828       __unwind$49498             0010c828 f   SW_Registrykey.obj
 0001:0000b984       __unwind$49790             0010c984 f   SW_Registrykey.obj
 0001:0000bb64       __unwind$49901             0010cb64 f   SW_Registrykey.obj
 0001:0000bb84       __unwind$49902             0010cb84 f   SW_Registrykey.obj
 0001:0000be44       __unwind$50129             0010ce44 f   SW_Registrykey.obj
 0001:0000be64       __unwind$50130             0010ce64 f   SW_Registrykey.obj
 0001:0000be84       __unwind$50131             0010ce84 f   SW_Registrykey.obj
 0001:0000bf8c       __unwind$54104             0010cf8c f   Utilities.obj
 0001:0000c820       ?FixupDialogItem@@YAXPAUHINSTANCE__@@PAUHWND__@@PAUDLGITEMTEMPLATE@@PAG3@Z 0010d820 f   Utilities.obj
 0001:0000ec34       doexit                     0010fc34 f   corelibc:crt0dat.obj
 0001:0000f210       ?CanThisExceptionObjectBeDestructed@@YAEPAUEHExceptionRecord@@E@Z 00110210 f   LIBCMT:frame_ce.obj
 0001:0000f55c       ?CallCatchBlock@@YAPAXPAUEHExceptionRecord@@PAKPAU_CONTEXT@@PBU_s_FuncInfo@@PAXHK@Z 0011055c f   LIBCMT:frame_ce.obj
 0001:0000f8f4       ?BuildCatchObject@@YAXPAUEHExceptionRecord@@PAKPBU_s_HandlerType@@PBU_s_CatchableType@@@Z 001108f4 f   LIBCMT:frame_ce.obj
 0001:0000fac8       ?FindHandler@@YAEPAUEHExceptionRecord@@PAKPAU_CONTEXT@@PAU_DISPATCHER_CONTEXT@@PBU_s_FuncInfo@@H@Z 00110ac8 f   LIBCMT:frame_ce.obj
 0001:00010430       ??__EgCommandCS@@YAXXZ     00111430 f   ModemStat.obj
 0001:00010454       ??__Eg_objModemStatus@@YAXXZ 00111454 f   ModemStat.obj
 0001:00010474       ??__Eg_Log@@YAXXZ          00111474 f   SW_Log.obj
 0001:00010494       ??__EtheSWIDisplayRawDataCR@@YAXXZ 00111494 f   SW_Log_Include.obj
 0001:000104b8       ??__E_AtlBaseModule@ATL@@YAXXZ 001114b8 f   atls:atlbase.obj
 0001:000104f4       ??__FgCommandCS@@YAXXZ     001114f4 f   ModemStat.obj
 0001:00010510       ??__Fg_objModemStatus@@YAXXZ 00111510 f   ModemStat.obj
 0001:0001051c       ??__Fg_Log@@YAXXZ          0011151c f   SW_Log.obj
 0001:00010528       ??__FtheSWIDisplayRawDataCR@@YAXXZ 00111528 f   SW_Log_Include.obj
 0001:00010544       ??__F_AtlBaseModule@ATL@@YAXXZ 00111544 f   atls:atlbase.obj
